:106EF300FF4DFF4DFF4DFF4DDF55FF5DFF5DFE5E17
:106F03001E5E1E5E1F561F561F4E1F4DFF4DDF4D4B
:106F1300DF4DDF4DDF4DBF4DBF4DBF4DBF4DBF4DAE
:106F2300BF4DBF4DBF4DBF4DBF4DBF4DDF4DDF4DBE
:106F3300DF4DDF4DDF4DDF4DDF4DDFEFBFEFBEEF49
:106F4300DFC73E757A555B4D7C4D7C4D5D4D5D4D88
:106F53005C5D9D65DE965DD7BFF7BFF79EF7BEEF1D
:106F6300BFEFBFEFBEE7FFA71E6E1D6E1E7E3F86FF
:106F73003E865F8E3FA65EDF7FF7DFF7BFF7BFF783
:106F8300BFF7DFD75FA63C965E865F8E7F965EB6C1
:106F9300DEE7DFEFBEEF9DEFBFCF7F85FC75DE6DD4
:106FA3009E755CBEFFEF9FE79EDFDF9EBD551A55C2
:106FB3007C557B969DD7FFDFBFD79F961D7DDE7DDA
:106FC300FEB73FDFDFD79FA65C7D9B8E1CBF5FD7DD
:106FD300BFAEDD85DB8E3D863D863E969F9E7FA6BA
:106FE3009FB6DFAE9F9E3D961D8E1E861E861E8516
:106FF300FE8E1F8DFF8E1E963EA69E96FF661C5527
:10700300FC561D561D561D5DFD763D9E9EAEDFAEA4
:10701300DFB6BEBEDFB69EB6BEC6FFCF1FD75FD7F5
:107023007FD73FD75FD75FDF7FDF7FD73FCF5FCF8D
:107033005FBF1FB6DFA67E8E5E7E3E761E6E1E6629
:107043001E661E65FD6DFD863D969F8E3E8E1D8ED2
:107053001D9E7EA6BFA6DFA6BEAE9EAEBEA6DE9ECC
:10706300FFA71FAF1FB71EB71EB71FAF1FB71FB7AF
:107073001FBEFFBEDFB6FFB6FEBF1EC6FEC6DEBE28
:10708300DFAEDFAEDFAEBFA6BFA6DFA6BFA6DFA61D
:10709300BF9EBF9EDF96DF96BF8E7F865F867F761D
:1070A3003E65FD5DFD55DD55FE55DE4DFE4DFE4D48
:1070B300FE55DE55FE55FE5DFD6E7E7EBE86DE769A
:1070C3009E663E661E5DFE55DE5E1F561F55FF55CE
:1070D300FF561F4E1F4E1F561F561F5E1E5E1F5E1E
:1070E3003F5E3F5E3F5E3F563F561E55FE4DDF4DB2
:1070F300DF4DDF4DDF4DDF4DDF4DDF4DDF4DDF4D2D
:10710300DF4DDF4DDF4DDF4DDF4DDF4DDF4DDF4D1C
:10711300DF4DDF4DDF4DDF4DDF4DDFFFFFFFDEF7DF
:10712300FFC7BF6DFD55BD4DBE4D9E4D7E559E5552
:107133007D5DBE65BD85FCCF9FEFFFF7BFF7DFEF3A
:10714300DFE7DFEFDFE7FFC79F8E5D865D863D8666
:107153001D863E761D7DDBAEFDCF9ECF9ECF7ECFBF
:107163007ECF7EC75E8E1A7DDA7DDC7DFC85DB8E6D
:107173001BBF5ECF7ED77FCF5FBF5F9E9D85FB86A4
:107183001C7DFCA6BEB73EA6DD9EFE96BE8DFC868C
:107193003C865D8E7D9EBE9E9E9E9E96BEA75FBFD5
:1071A3003FB71E9E7C967DA6BEC75FD75ECF1CAE43
:1071B300BBAE9BB71DBF7FAF1E965E967F961E9E8E
:1071C3001EAE7EBEFFBEDFB6BEAEBE963D85FE7D65
:1071D300DD85FE8E3E8E3F965F9EBF96DF765F66B1
:1071E3001E663F665F665F663F6E3F7E3E8E7F969E
:1071F3009F9E9EA69EAEBEAEDFAEBEAE9EB69EB6B2
:10720300BEBEFFC71FC6FEC6DECEDECEFFC6DEBED7
:10721300BEB6BFB6DFAE9F9EDF8E9F865E867F863D
:107223007F867F8E9F969EA6DFA6DFAEFFAEFFB75B
:107233001FBF3FC73FC73FC73FCF1FC73FBF3FB773
:107243003FBF1FBEFFAF1EAF1EAEFEAEFEA6DEA645
:10725300BEAEBEA6DFAEDFAE9DC6DDE79FCF1EA6E8
:107263009E969F8E7F8E9F867F7E5F7E5F765F6E0C
:107273001F661E5E3E663E663F665F665F5E3F5606
:107283001E4E1F4E1F4E1F4E1F4E1F4E1F4E1F4D95
:10729300FF4DFE563F5E5F5E5E667E665E661D5513
:1072A300FD4DDE4DDE4DDE4DFF4DFF4DFF4DFF4DE0
:1072B300FF4DFF4DFF4DFF4DFF4DFE4DFE4DFF4D6D
:1072C300FF4DFE4DFE4DFE55FE55FE55FE4DFF4D49
:1072D300FF4DFF4DFF4DDF4DDF4DDF4DDF4DDF4DEB
:1072E300DF4DDF4DDF4DDF4DDF4DDF4DDF4DDF4D3B
:1072F300DF4DDF4DDF4DDF4DDF4DDFBEBCBEFDAEED
:10730300FD9F1E8EDE96BD9EBEA6BEA6BEAEDEAEA3
:10731300DEB6FEB6FEAF1EA6DE9E9DA6BEAEBDAE1B
:10732300BDA6BDA6BDAE9DAE9DC77FD79FDFBFDF08
:10733300BFDFBFE79FE7BFD75DB6BC9E9D8E5D7E77
:107343003D7E1C7DFBB73EDFDFDF9FDF9EDFBFD7C8
:10735300DF869D65FC763E761F6DBD96BECFFFD75B
:10736300BEDFBECFDF867C4DBC4DDF559D96DED79D
:10737300FFDF9EDFBF967E559D4DDD5DDBB77EDF74
:107383009EDF9FB69CAE7BD75EF7FFFFFFF7DEE77E
:107393009EDF7EC6DBD77ED7BFAE9DA63DA65EA68B
:1073A3005DAE5DB69EB6BEBF1FC75FAEDE8E5E9698
:1073B3005E967F969F967E967E8E3E865E7E5E76F8
:1073C3005E661D6E1D6E5E765F763E763E867E96AB
:1073D300BE969E9E9E9E9E9EBEA6BFA6BFA6BFA60F
:1073E3009EA69EA69E9E5DA67DA67EA69EA69F9E0B
:1073F3009E9E9F969F969F967E8E7E8E7E967E966F
:107403007E969E9EBE9EBFA6BFA6DF9EDF9EDF9694
:10741300FF9EFE9EDE9EDE9EBF9E9E9E9E96BF8E1E
:107423009F969F9E5E865F867F8E5E965E9E7F9E04
:107433009F9E9F969F969EAEBECF5FCF7FA6BE7E3A
:107443005E6E3E5E1E561E561E561E4E1E4E1F4E30
:107453001F461F4E1F4E1F4E1F4E1F4E1F461F46D9
:107463003F4E3F4E1F4E1F4E1F4E1F4E1F561F4E69
:107473001F463F463F4E3F4E1F4DFF4DFF4E1F4E93
:107483001F4E1F4E1F4E1F4E1F4E1F4E1F4E1F4699
:107493001F4E1F4DFF4DFF4DFF45FF45FF45FF4D60
:1074A300FF4E1F563F5E3F5E5F665F5E3F561F4E59
:1074B3001F4DFF4DFF4DFF4DFF4DFF4DFF4DFF4D49
:1074C300FF4DFF4DFF4DFF4DFF4DFF4DFF4DFF4D59
:1074D300FF4DFF4DFF4DFF4DFF4DFF43B44CB95DD5
:1074E3007D6DBBCF7FF7FFFFFFFFFFFFFEFFFFFFBA
:1074F300FFFFDFF7DFE7FF8E7D559C5E1E65FE769F
:107503001E7E3E7E5F863E963DDFBFEFFFF7FEFFAA
:10751300DEFFBFF7BFF7DFEF9FCEFEBEDFAEBFB626
:10752300BFBF1FAEFFBEFEEFDFF7BEF7BEEFBEEF7E
:10753300FFAF7F559C55DE4DFF4DDE65DCBF5EE73B
:10754300DEEF9DDFBEBF9F6E1D55FE5DFD6E1BB75B
:107553007FCF9FCFBEBFBF8E9D7E3D965CC6FDEFA6
:10756300DFEFDFF7FFFFFEFFBEFFBEF7DFF7FFFF33
:10757300DEFFFFEF9EE77ED77ECF5FBF1FBF1FBE3D
:10758300FFBEFFA67EA67EAEBFA69E9E5DA69EA65E
:10759300BEAEDEA6BE9E7D9E7E9E7E9EBE9EBE9E91
:1075A300FE9EDE96BD9EDE9EDE9EBE969E9EBEAE79
:1075B300DFB6DEB6FFB6FFB6FFAEDFAEDFAEFFAEC1
:1075C300FFAEFFAEFFAEDFAEDFA6DFA6BF9EBF9E60
:1075D300BF96BF969F969F967F9E9FA6BFA6BE9E71
:1075E300BE9EBE9EBE969E869E763E661D5E1D5EBA
:1075F3001E5E1D5E1D5E1D5E1D6E5D663D563D5627
:107603003E5E1E6DFD761D75FC8E5DA6FF96DF86C4
:107613009F6E7F663E867E9EFF9E9F7E1D5DFD560E
:107623001E4E1E4E1E4E3E4E3F4E3F4E3F4E3F4E53
:107633003F463F4E3F4E3F4E3F4E3F4E3F4E3F4EE7
:107643003F4E3F561F4E3F4E3F4E3F4E3F4E3F4EE7
:107653003F4E3F463F4E1F461F461F4E1F4E1F4E77
:107663001F4E1F4E1F4E1F4E1F4E1F4E1F4E1F4DB0
:10767300FE4E1F561F55FE5DFE5DFE55FE4DFE4E32
:107683001F4DFE4DFE561F4DFF4DFE55FF4DFF4D49
:10769300FF4DFF4DFF4DFF4DFF4DFF4DFF4DFF4D87
:1076A300FF4DFF4DFF4DFF4DFF4DFF4DFF4DFF4D77
:1076B300FF4E1F4E1F4E1F4E1F4DFF95BA54155CB4
:1076C300779E3DDF7FF7DFF7DEF7DEF7DEF7BEF706
:1076D300DFF7DFF7BEF7DFAEBD5DDD561F561F5D7B
:1076E300FF6E1F6E3F661F7DFDB71EE7FFEFDEF7E0
:1076F300DEF7BFF7BEEFDFEFDFBEBDA65DA67DA65B
:107703009DAEBDAE3CAE3BD79FD7DFCFBFCFBFD77C
:10771300BFB75F8E9D8EBD86DE86DE8E9DAEFEB7C5
:107723001FAF1FA6DEA69DB75EBF5EBF5EC77E9E70
:10773300BD7E1C865C9E9CC73EE79FEFBFF7BEFFE6
:10774300BDF7DFEFBFF7BFFFDFFFDFFFDFFFDFFFC8
:10775300DEF7DEFFFFEFFFD73EBEFEBF3EB71FB62D
:10776300FEAEBEA67DAEDEAEBE9E5DA67DAE7CBE8B
:10777300FDD77FCF7EC71DC71EC73FCF3FCF1EC6D6
:10778300FEC71FC73FC71FC71FC73FC73FC71FC787
:107793003FCF3FC71FC71FC71FBF1FB6FFB6FFB6E9
:1077A300FFAEFFAEDFAEDFA69EA69EA69EAEBEAE2A
:1077B300DFAEDFA6BEA6BEAEBFAEDFAEFFAEFEA699
:1077C300FFA6FF96BF7E5E6E5F665E563F4E3F4EE0
:1077D3003F563F563F65FCA6FDBFBF869C65DA86D4
:1077E3003CAEFEC75FD77FCF3ED77FC77F9E9E7ECF
:1077F3001D6E3E5DFD6DFD7E3E75FE661E563F4E63
:107803003F463F4E1F4E1F4E1F4E1F4E1F4E1F4ED5
:107813001F4E1F4E1F4E3F4E3F4E1F4E1F4E1F4EBD
:107823003F4E3F4E3F4E3F4E1E4E1E463E3E3E4651
:107833005E563E5E3E665E6E5E6E5E665E5E3E4EAD
:107843003E4E3E4E3E4E1E4E1E4E1E4E1E4E1E4E75
:107853001E5E3F667F6E9F767F6E7F663E561E4E30
:107863001F4E1F4DFF4DFF4DFF4DFF4DFF4DFF4D74
:10787300FF4DFF4DFF4DFF4DFF4DFF4DFF4DFF4DA5
:10788300FF4DFF4DFF4DFF4DFF4DFF4DFF4DFF4D95
:10789300DE55DE55DE55BE4DDF4DFF957895578499
:1078A300B49D16E75EFFFFF7DFFFDFFFFFFFFFFF7C
:1078B300FFFFFFF7DFF7FFCF3E965D763D661D6E58
:1078C3001D761D763D7E5E861CA6DDD79FDF5FE7B6
:1078D3007FE77EEF7FEF9FEF9FE7BFDF7ED75ECF30
:1078E3003ECF5EC73DC75EA6DD7E1C661D663D6E50
:1078F3001C6DDBA71DE7FFF7DEF7BEEFFFC79F7E1B
:107903001D763E867F8E5DCF7FEFFFEFBFEFDFCF2C
:107913009F9E9D9E7E9E9EB6DDDFBFF7BFFFBFFF8E
:10792300DEFFDFFFDFFFDFFFDFFFDFFFFFFFDFFF45
:10793300BEF7BDEFBEE79ECEDDDF5EDF9EB6DDB6F2
:10794300DDD75ED73DE7BFDF9FCF5ED77ED75EEF44
:10795300FFF7FFFFFFFFFFF7DEF7FFF7DFEFBFDF05
:107963005EDF7ECF1EBEFEB6DDB6DEB6FEBF1FBF38
:107973001FBF1FBEFEBEFEBEDEBEFFB71FB6FFB6F5
:10798300FFB6FFBF1FB6FFB6DEB6DDB6DEBF1EC74E
:107993003FC73FC73FC71EBEFEBEDEB6DEB6FFAE65
:1079A300FF969E7E5E767E765E6E5E6E7E6E5E6E0B
:1079B3005E6E5D6E5D7DFACF3ECF5F8E5B8E9BCF3D
:1079C3007FF7DFEFDFEF9FE77FD75FB6BD9E7D9E3B
:1079D300BF867E863D967E9EBF9EDF96DF869E7621
:1079E3005E6E7F6E7F667E667F665E5E5E5E7E5ED9
:1079F3007E5E7E5E5E5E5E5E7E567F567F565F5621
:107A03005E563E5E5E6E3D869E8EBE869E7E9F76F3
:107A1300BF767E7E9E867E8E7E867E767E665D5673
:107A23005D563E5E3E5E3E5E3F563E563E565E565B
:107A33003E5E3E5E3E5E5E5E5E563E5E3E565E4E23
:107A43005E563E563E561E563E563E4E3E563E569B
:107A53003E563E563F4E1E4E1F4E1F561F561E5637
:107A63001E563E4E3F563F563F561F5DFD763D9692
:107A7300DEA6FEA6FF96BF7E7E663FBE5ABE5ACEE8
:107A83009BADB89D15BE3AE7BFDF5ED73ECF3EC67E
:107A9300FEBEDEB6BDBE9DCF1EDF9FD79ECF7ED777
:107AA3009ED79EDFBFE7BFE7DFDF7EBE5CBE5DBE66
:107AB3009EC6DFCEDED6FEC69DD6FDF7DFF7DFFF1F
:107AC300DFFFFEFFFFF7FFCF7F861C763E661F6555
:107AD300FE7DDCAEBCE7DFEF9EF7BFEFDFDFFFA687
:107AE300DE7E1D863E965DAEBCDF9FDF9ED77ECFDA
:107AF3007EBF5EC75ECF3ED75EEFBFFFDFFFBFFF38
:107B0300DFFFDFFFDFFFDFFFDEF7DFF79FEF9FF72B
:107B1300FFF7FFEFDFD6FDCEDDE79FEFDFE79EEF59
:107B23009FF7DFFFFFFFFFF7DFF7DFEFDFEFDFEFAA
:107B3300BFF7DFFFDEFFDEFFFFFFDFFFDFF7BFF78C
:107B4300BFF7BFE79FE7BFD75EC6FDB6DDB6FDBF94
:107B53001EBF3EBF3EBF1EBF1EBF1EBEFEBEFEBE3D
:107B6300FEBEFEC71EC71EC73ECF5FCF7FCF5FCF10
:107B73003ECF3EC71EC71EC71EBF1EBF1EBF1EAEC3
:107B8300FDA6DD9EBC9EDD9EFDA6FDA6FD9E9CAED4
:107B9300FDBF5ECF5ED77EDF5EDF7ECF9FAEDCC6EE
:107BA300FDE77FDF5ECF3ED77EBEFDB6FDBF1EBFC6
:107BB3003EB6FEB6FEB71EAEFEAEFDA6BCA6BCA686
:107BC300DD9EDD96BC96BC96DD96BD8EBC8EBC8ECE
:107BD300BD8EBD8EBC86BD86BC86BC86BC8EBC8E6F
:107BE300BC96BCA6DDAF3EB75EB71DB6FDAE9CAE80
:107BF3009C9EBC9EBC9EBC8E5B965CAEFDB71EAECF
:107C0300FEA6FE96DD7E9C7EBD76BD7E9D7E9D7628
:107C13009D769D769D769D769D769D769D769D7EC1
:107C23009D86DD86BD86BE7EBE769D6E9D6E9D6EF7
:107C33009D6E9D6E7D6E7D6E7D6E7D6E7D667D66B9
:107C43007D667D667D667D6E5C769DA71EBF3FB6B5
:107C5300FEBF3FB73F9EFE86DE769E8D168D168C49
:107C6300F68D169538324D5BD39DDB95FC8DDC8507
:107C7300DD7DFE861E85FD9E3DE7BFFFFFFFDEFF28
:107C8300DEFFFFFFDEFFDDFFDEEFBFB65DA63EA634
:107C93007F9E5FA65EAE7EAE5DB65BE79EF7DFF7C7
:107CA300DEFFDEFFDEF7DFDFBFAE9DA69DA6BFAE24
:107CB300FFCF5FDF9FE7BFEFBFEFBFEFDFE7BEDFC2
:107CC300BFD77FCF5FDF9FE7BFE79ECF1DBEFDAE70
:107CD3007CBEDCE7DFF7FFFFDFFFDEF7BFF7BFFFA9
:107CE3009FFFBFFFDFF7DEF7FFE77ED6BDD6DDDF01
:107CF3005FDF9FD77ED75EDF5DEF9FEF7EF7BFFF2E
:107D0300DFF7BEFFBEFFDFF7BFEFBFE77FEF7FEF1A
:107D13009FF7BEFFBEFFBEFFBFF7BFF7BFF79FEFE3
:107D23009FE75EDF3EE79FEFBFDF9FC73FC73FC7CA
:107D33003FC73FBF1EC71FBF1FBF1FB6FFB6DEB67D
:107D4300DEB6DEB6DEB6DEB6DEAEDFB6FFB6DEAE7E
:107D5300BEAEBEB6BEB6DFB6FFAEDFB6DFAEBEAEFC
:107D63009DAEBDB6BDC73EE7BFE79FCF1DCEFCDFCF
:107D73005EEFBFF7DFFFDFF79EE77EE7BFC6DDBE3F
:107D83009DC6FEC6BDB6BEAEBE9E7D967D967D9655
:107D93005D967E8E5E8E3E8E1D8E3D9E7D9E7DA665
:107DA3009DA69D967D969D8E5D7E1C7E3D8EBE8698
:107DB3009E7E3E761E763E763D763D7E5E865E9662
:107DC3009EAEBFAEBF9EDF8E9E7E5C75FB7E3CA6E5
:107DD300BEBEBEBEDFAEFF9EBE9EBEAF1EB6DEA65D
:107DE300BE8E9E765D563D4E5D4E3D4E1E55FE4EFD
:107DF3001E4E1E4E1E4E3E4E3E4E1D4E3E5E1D6E92
:107E03003D767E7E7E765E663E5E1D561D561D5613
:107E13001D561E561E561E55FE5E1E5DFF5DFE5E02
:107E23001E5E1E661E6E1E6DFE7E3E867E863E7D39
:107E3300FD75DC6DDC5DBC55DD661E63F464147496
:107E4300766C55957A4331222D2AB0649785FE7E50
:107E53001E75DE75FE75DE963DD79FF7DEFFDEFFEE
:107E6300DFF7DFF7DEF7DEF7FFE7FFBEDEA67EA66E
:107E7300BF9E7EAE7EB6BEB6BEBEBDD75EDF9EDF04
:107E83009FDF7FD75ECF3FC71ED73EE79EF7BEF784
:107E9300BFF7DFEFDFE77ED71EDF3FE75EE75DE794
:107EA3005DFFBEFFFFFFFFFFFFF7DFE7BFC71EBE9C
:107EB300DED73EEFBFFFFFFFDFFFDFFFDFF7DFF7B9
:107EC300BFF7BFF7DFEFBFE79FD71EDF7FE79FDF78
:107ED3005EBE9DAE5DBEBDE7DFF7DFF7BFF79FF781
:107EE300BFEFBFEF9FE77FDF5FD73FCEFEDF3FEF01
:107EF3007FF7BFF7BEEF9EEF9FE77FDF7FD73FC6DA
:107F0300FEC6BEC6FFC71FC73FBEFEB6DFBEFFBF6E
:107F13001FBEFFB6FFB6FFB6FFAEFFA6FFA6DFA6E6
:107F2300DFA6DFA6DFA6DFA6DF9EBF9EBF9EBF9EA6
:107F33009FA6BFA6DFA6BFA69EA69EAEBFA69EAE69
:107F43009EBEDED77FE7BFEF7FEF5FEF7FEF9FE759
:107F53007FE75EE77EEF7EEF7EDF7EDF5FDF5FC77B
:107F63005FBF3FAE9EA69F969F969F8EBF869E7EC7
:107F73007E869F867EA6BEB73FC75FCF9FCF5FCF6C
:107F83003FCF5FD77FCF5FCF5FBEFEBF1FB73FAE91
:107F9300DF9EDF8EDF8EBF86BF86BF869E867E8E88
:107FA3009F867E867E869E7E9E867E967EAEFFB66C
:107FB300FFC6DFB6BFA69EA6FF96FE8E9D8E7C8E65
:107FC3005D8E5E7E7E767E6E9F6E9F6E7F6E5F6E33
:107FD3005E6E7E665E663E665E665E6E7F6E7E6E1D
:107FE3005D6E3D6E3D6E5E6E5E6E7E667E6E7F6E18
:107FF3005E6E5E6E5F6E5F6E3F6E5F6E5F765F7628
:108003007F769F769F767F7E7F7E7F7E7F7E9F7E3D
:108013009F7E9F7E7E7E7F867F8EBF84D784B6635E
:10802300927C55ADDB4B303ACF2A8E1A4D3B5275BD
:108033007B865E8E5E965FAE9DD79FF7FFF7DFF779
:10804300DFF7DFEFDFDF9FDF9ECF5EBEDDBEDDC686
:10805300FDD73EDF7EE79FE79EE7BFCEFDAE3CB692
:108063009EAE7E9E5D9E9F8E1DBEFEF7FFFFBEFFF2
:10807300BEFFDEFFFFE79FC6BEC6DED73EEF7FEF44
:108083009FF7BEF7FFF7DFFFDEFFBEEF7ED71EDFF2
:108093007FEFBFEFBFE77EDF3EE75FE77FF7DFF707
:1080A300DFF7DFE7BFC6DEBE7DB65CD77FE7DFE77E
:1080B300DFBEBDA63DB69DCF5EDF7EF79FF7BFF760
:1080C300DFE79FD73ECF3FC71FC6DFC6FFCEFFD731
:1080D3003EDF7EE79EE7BFD73EBEBEAEBE9E7E9E20
:1080E3005E9E5F9E7F9E7F9E7E9EBF9E9F9E9F9E67
:1080F300BF9EBF969E969E969E9EBEA6BEA6BEA6FB
:10810300BEA6BEA6BEA6DEA6BEA6DEA6BE9E9E9E3C
:108113007DA6BFAEDFA69EA69EA6BEAEFFA6BFAE41
:10812300BFBEFFC6FECF1ECEDDC6DDCF1ECF1FD71F
:108133001FDF1EE75EE75FD73FBEFDC6DEC6DFAECD
:10814300FF9EBF9E7F967E969E8E9E8EBF8EBF8E17
:108153009F96BF96BFA6DFB71FB6FFB6DEBEDFBED4
:10816300DFBEDFBEDEBEFFB6FEAEFFA6DF965D8ED0
:108173007E8E9E869F869F7E9F7E9F7E9E7E9F7E17
:108183007F769E7EBF7E7F867F8E7F969FA6BE9ED6
:108193009D8E9E969E9E9E9EBFA6BFAEDFAEFFAEF9
:1081A300FFAF1FAF1FB71FAEFFAEFFAEFEA6FEAE03
:1081B300FFAF1FAEFFAEFFAEFFAEFFAEDFA6FF9E6B
:1081C300FFA6DFA6BFA6DFA6BF9EBF9EBF9EBF962C
:1081D300DF96BF8EBF86BF869E7E9E765E765F6E7F
:1081E3005F6E5E665E663E661E6E3F6E5E6E5E6EC2
:1081F3005E767F765E765E7E7E7E5E533042AE082E
:1082030086426D8C956BD263F36C754B921A2D324B
:10821300F08DBBA69EBEDDC6FDD75EDF5EDF3EDF13
:108223003EDF3DD71DC69DBE9CAE3BBEDDEFFFF7D7
:10823300FFFFFFFFFFFFDFFFFFF7FFD73EAE7DAE80
:108243009F963E8E3F863F85FDA65DE7BFF7DFF72E
:10825300DFF7DEF7DEEFDFC6DDBE7DCEDDDF1DE758
:108263003EE77EE7BFE7BFE79FEF7EF7BFF7FFF786
:10827300DFF7DFEFFFC6BCBE5CC6BEBE9DDF7FEF90
:10828300DEEFDFDF9FB65CAE3CAE1BB6DDC73EBEA6
:10829300FEB6BECF3FDFFFCF7DCEFDDF3FEF7FF7E3
:1082A300DFE79FCF1EC6FFBEDFB6BEBEBEBEBECFDC
:1082B3003FDF7FDF9FE7BFCEFDB63B961D8E3E8E31
:1082C3003E8E3E967F969F9EBF9EBF9EBE9EBF9E46
:1082D300BF9EBF9EBE96BE9EDFAF1FB71FBF3FBFF1
:1082E3005FBF3FC75FC75FC73FC73FC75FC75FC7C3
:1082F3005FBEFEB6DFB6DFB6DFB71FAEDFAEDFB6FB
:10830300FFBEDFC6FEC6FEC71EC71EBEFEC6FFCF2C
:108313001FDF5FE77FDF5FC73FAEBEA65CAE9E9EFB
:108323007E8E7E967E969D969D8EBE96DE96BE969C
:108333009E9E9F9EBF96BF969F969F967E965E96A5
:108343007F967F967E967E8E5E8E5E865E869F8607
:108353009F869F8E7E8E7E867E867E867E869E8688
:108363009F7E9E7E9E7E7E867E867E869E7E7D868A
:10837300BE86BF869F8EBF8EBF8E9F8EBF86BF8EEB
:10838300BF8EDF8E9F969F8E7E8E5E865D7E5D8620
:108393005D865D8E9E96BE9EDF9EFF96DF96DF9680
:1083A300DF96BF96BF969F9E9F9EDF9EDFAEBFAEBA
:1083B300DFAEDFA6DFA6DF9E9F8E7F865F765F6ED2
:1083C3005F663E663E663E663E6E1F661E663F6E97
:1083D3005F6E7F665E665E6E5E6E3E07E007E00779
:1083E300E007E007E007E007E007E007E007E00752
:1083F300E007E007E007E007E007E007E007E00742
:10840300E007E007E007E007E007E007E007E00731
:10841300E007E007E007E007E007E007E007E00721
:10865300E007E007E096B6BE3A773207E007E007A7
:10866300E007E007E007E007E007E007E007E007CF
:10867300E007E007E007E007E007E007E007E007BF
:10868300E007E007E007E007E007E007E007E007AF
:10869300E007E007E007E007E007E007E007E0079F
:1086A300E007E007E007E007E007E007E007E0078F
:1086B300E007E007E007E0478DB5FAADF9C61AB663
:1086C30079675107E007E007E007E007E007E00705
:1086D300E007E007E007E007E007E007E007E0075F
:1086E300E007E007E007E007E007E007E007E0074F
:1086F300E007E007E007E007E007E007E007E0073F
:10870300E007E007E007E007E007E007E007E0072E
:10871300E007E007E007E007E007E07EF3BDDAAD3E
:10872300F9ADF9B5F9C61BAE98576F07E007E00737
:10873300E007E007E007E007E007E007E007E007FE
:10874300E007E007E007E007E007E007E007E007EE
:10875300E007E007E007E007E007E007E007E007DE
:10876300E007E007E007E007E007E007E007E007CE
:10877300E007E007E007E007E007E007E007E0AE17
:1087830058B5D9ADD9ADD9ADD8ADF9B5D9C5FB9EDD
:10879300D63FAD07E007E007E007E007E007E007A3
:1087A300E007E007E007E007E007E007E007E0078E
:1087B300E007E007E007E007E007E007E007E0077E
:1087C300E007E007E007E007E007E007E007E0076E
:1087D300E007E007E007E007E007E007E007E0075E
:1087E300E05F4FBDFAADD9B5D9B5D9ADF9ADD8CEA6
:1087F300BBC67ABDB9C61A8EF42FAB07E007E007F4
:10880300E007E007E007E007E007E007E007E0072D
:10881300E007E007E007E007E007E007E007E0071D
:10882300E007E007E007E007E007E007E007E0070D
:10883300E007E007E007E007E007E007E007E007FD
:10884300E007E007E08EB5B5DAADF9ADD9ADD9B53E
:10885300F9ADD8D6BBF7DFE73CBE19BDDAB6597F11
:108863001207E007E007E007E007E007E007E0079B
:10887300E007E007E007E007E007E007E007E007BD
:10888300E007E007E007E007E007E007E007E007AD
:10889300E007E007E007E007E007E007E007E0079D
:1088A300E007E007E007E03FACBE19ADD9B5D9ADAD
:1088B300D9ADD9ADD9ADD9ADB8BE19E73DFFDFD636
:1088C300FCB5F9C5FBBE796F5107E007E007E00788
:1088D300E007E007E007E007E007E007E007E0075D
:1088E300E007E007E007E007E007E007E007E0074D
:1088F300E007E007E007E007E007E007E007E0073D
:10890300E007E007E007E007E007E07712BDDAAD34
:10891300D8ADD9ADD9ADD9ADD9ADD9ADF9ADD8AD06
:10892300B8C65ADF1CADF9ADF9B5FAC61BAE984708
:108933008D07E007E007E007E007E007E007E0074F
:10894300E007E007E007E007E007E007E007E007EC
:10895300E007E007E007E007E007E007E007E007DC
:10896300E007E007E007E007E007E007E007E0A62D
:1089730057B5D9ADF8ADD9ADD9ADD9ADD9ADD9AD1F
:10898300D9ADF9ADF9ADD8ADB8ADD9ADD9ADD9AD96
:10899300F9BDFAAE3807E007E007E007E007E007B4
:1089A300E007E007E007E007E007E007E007E0078C
:1089B300E007E007E007E007E007E007E007E0077C
:1089C300E007E007E007E007E007E007E007E0076C
:1089D300E0576FBDDAADD9ADF8ADD9ADD9ADD9ADED
:1089E300D9ADD9ADD9ADD9ADD9B5F9B5F9ADD9AD04
:1089F300D9ADD9ADF8AD98963507E007E007E007A4
:108A0300E007E007E037A96EC907E007E037A907E9
:108A1300E007E007E007E007E007E007E007E0071B
:108A2300E007E007E007E007E007E007E007E0070B
:108A3300E007E007E08EB4BDDAADF9ADD8ADD9AD4E
:108A4300D9ADD9ADD9ADD9ADD9ADD9ADD9ADD9ADF3
:108A5300D9ADD9ADD9ADD9ADD8B5785F0F07E0079A
:108A6300E007E007E007E007E0CE248E4707E09643
:108A73006607E007E007E007E007E007E007E00735
:108A8300E007E007E007E007E007E007E007E007AB
:108A9300E007E007E007E037ACB619ADD9ADF9B5AB
:108AA300D9ADD9ADD9ADD9ADD9ADD9ADD9ADD9AD93
:108AB300D9ADD9ADD9ADD9ADD9ADF9ADB8ADD7072C
:108AC300E007E007E007E007E05F0907E0BD649C1B
:108AD300A56728F5025E8807E007E007E007E007DF
:108AE300E007E007E007E007E007E007E007E0074B
:108AF300E007E007E007E007E007E06F11BDDAAD4C
:108B0300F8ADD9ADD9ADD9ADD9ADD9ADD9ADD9AD13
:108B1300D9ADD9ADD9ADD9ADD9ADD9ADD9ADF9B5FA
:108B2300797E9307E007E007E007E09EA68E6707DC
:108B3300E075C807E04749AC6436C807E007E007BB
:108B4300E007E007E007E007E007E007E007E007EA
:108B5300E007E007E007E007E007E007E007E0A63B
:108B630077B5DAADD9ADD9ADD9ADD9ADD9ADD9AD2B
:108B7300D9ADD9ADD9ADD9ADD9ADD9ADD9ADD9ADC2
:108B8300D9ADD8AD98476D07E007E007E007E0C52A
:108B9300C5CC6307E007E007E0470907E007E00704
:108BA300E007E007E007E007E007E007E007E0078A
:108BB300E007E007E007E007E007E007E007E0077A
:108BC300E0476DBDFAADF9ADD9ADD9ADD9ADD9ADEC
:108BD300D9ADD9ADD9ADD9ADD9ADD9ADD9ADD9AD62
:108BE300D9ADD9ADF9AD989E3607E007E007E03F70
:108BF300A907E085A83E6807E0A685AE0607E0075B
:108C0300E007E007E007E007E007E007E007E00729
:108C1300E007E007E007E007E007E007E007E00719
:108C2300E007E007E086D4BDDAADD8ADD9ADD9AD64
:108C3300D9ADD9ADD9ADD9ADD9ADD9ADD9ADD9AD01
:108C4300D9ADD9ADD9B5D9ADF9B57966F007E00796
:108C5300E05F476EA807E0378A07E007E0A606CC87
:108C63002307E007E007E007E007E007E007E00786
:108C7300E007E007E007E007E007E007E007E007B9
:108C8300E007E007E007E02FCBB618ADD9ADF9B5A3
:108C9300D9B5D9B5D8B5D8B5D8ADD8ADD8ADD8AD87
:108CA300D8ADD8ADD8ADD8ADD8B5D8ADD8ADD73708
:108CB300AB07E007E0DDE4B58507E007E066E82FF2
:108CC300AA6E082EE907E007E007E007E007E007E0
:108CD300E007E007E007E007E007E007E007E00759
:108CE300E007E007E007E007E007E06F11BDDAAD5A
:108CF300D8ADD8B5D8B5D8B5B8B5D8B5B8ADD8AD61
:108D0300D8ADD8ADD8ADD8ADD8ADD8ADD8ADD8B530
:108D130098869307E007E007E0A5667D0507E06F07
:108D230027CDC407E007E007E007E007E007E00717
:108D3300E007E007E007E007E007E007E007E007F8
:108D4300E007E007E007E007E007E007E007E09E51
:108D530056B5D9ADD8ADD8ADD8ADD8ADD8B5D8B551
:108D6300D8ADD8ADD8ADD8ADD8ADD8ADD8ADD8ADD8
:108D7300D8ADD8B578574E07E007E0378A5EAA0723
:108D8300E007E076E8E4024E8907E007E007E00742
:108D9300E007E007E007E007E007E007E007E00798
:108DA300E007E007E007E007E007E007E007E00788
:108DB300E0478DBDF9ADF9B5D9ADD9ADD9ADD9ADD3
:108DC300F9ADF9ADF8ADD9ADD9ADD9ADD9B5F9ADE9
:108DD300D9ADD9ADF8ADB895F507E007E007E007E1
:108DE300E007E007E007E06689560807E007E007C9
:108DF300E007E007E007E007E007E007E007E00738
:108E0300E007E007E007E007E007E007E007E00727
:108E1300E007E007E08ED4BDDAA5B8ADB8B5F9AD8B
:108E2300D9ADD9B5F9B5F9ADD9ADD9ADD9ADD9ADBF
:108E3300D9ADD9ADD9ADD9ADD9B5796EF107E007C3
:108E4300E007E007E007E007E007E02F8A07E00715
:108E5300E007E007E007E007E007E007E007E007D7
:108E6300E007E007E007E007E007E007E007E007C7
:108E7300E007E007E007E007E0AE38B5D98CB4A51A
:108E830077B5F9ADD9ADD9B5D9B5D9B5D9ADD9ADD1
:108E9300D9ADD9ADD9ADD9ADD9ADD9ADD9ADB83736
:108EA300AC07E007E007E007E007E007E007E007BB
:108EB300E007E007E007E007E007E007E007E00777
:108EC300E007E007E007E007E007E007E007E00767
:108ED300E007E007E007E007E007E05F30C5DAAD51
:108EE300D894D5B5D9ADD9ADD9ADD9ADD9ADD9AD65
:108EF300D9ADD9ADD9ADD9ADD9ADD9ADD9ADF9B517
:108F030099867407E007E007E007E007E007E0075A
:108F1300E007E007E007E007E007E007E007E00716
:108F2300E007E007E007E007E007E007E007E00706
:108F3300E007E007E007E007E007E007E007E09E5F
:108F430096B5FAA577A577B5F9ADD9ADD9ADD9ADB4
:108F5300D9ADD9ADD9ADD9ADD9ADD9ADD9ADD9ADDE
:108F6300D9ADD8B598574F07E007E007E007E0070A
:108F7300E007E007E007E007E007E007E007E007B6
:108F8300E007E007E007E007E007E007E007E007A6
:108F9300E007E007E007E007E007E007E007E00796
:108FA300E03F8DBDFAADF98CD4ADB8B5F9ADD9AD0F
:108FB300D9ADD9ADD9ADD9ADD9ADD9ADD9ADD9AD7E
:108FC300D9ADD9ADF9ADB9A5F607E007E007E007DC
:108FD300E007E007E007E007E007E007E007E00756
:108FE300E007E007E007E007E007E007E007E00746
:108FF300E007E007E007E007E007E007E007E00736
:10900300E007E007E07EF3BDDAA59794F5B5F9AD87
:10901300D9ADD9ADD9ADD9ADD9ADD9ADD9ADD9AD1D
:10902300D9ADD9ADD9ADD9ADF9B57976D207E007C8
:10903300E007E007E007E007E007E007E007E007F5
:10904300E007E007E007E007E007E007E007E007E5
:10905300E007E007E007E007E007E007E007E007D5
:10906300E007E007E007E007E0A637B5F994F5A5C8
:1090730077B5F9ADD9ADD9ADD9ADD9ADD9ADD9ADF7
:10908300D9ADD9ADD9ADD9ADD9ADF9ADB8ADB73F3E
:109093008C07E007E007E007E007E007E007E007E9
:1090A300E007E007E007E007E007E007E007E00785
:1090B300E007E007E007E007E007E007E007E00775
:1090C300E007E007E007E007E007E05F4FBDDAA550
:1090D300B78CB4ADD8B5F9ADD9ADD9ADD9ADD9AD9E
:1090E300D9ADD9ADD9ADD9ADD9ADD9ADD9ADF9B525
:1090F300998E5407E007E007E007E007E007E00781
:10910300E007E007E007E007E007E007E007E00724
:10911300E007E007E007E007E007E007E007E00714
:10912300E007E007E007E007E007E007E007E08E7D
:1091330095B5DAADD8A577B5F9ADD9ADD9ADD9AD7A
:10914300D9ADD9ADD9ADD9ADD9ADD9ADD9ADD9ADEC
:10915300D9ADD8B5785F2F07E007E007E007E00750
:10916300E007E007E007E007E007E007E007E007C4
:10917300E007E007E007E007E007E007E007E007B4
:10918300E007E007E007E007E007E007E007E007A4
:10919300E007E08E74B519ADB8ADF9ADD9ADD9AD71
:1091A300D9ADD9ADD9ADD9ADD9ADD9ADD9ADD9AD8C
:1091B300D9ADD9ADF9B5B99DD607E007E007E0070A
:1091C300E007E007E007E007E007E007E007E00764
:1091D300E007E007E007E007E007E007E007E00754
:1091E300E007E007E007E007E007E007E007E00744
:1091F300E007E007E007E007E06EB1A577AD38AD23
:10920300B8ADF9ADD9ADD9ADD9ADD9ADD9ADD9AD2C
:10921300D9ADD9ADD9ADD9ADF9B57976B207E007F6
:10922300E007E007E007E007E007E007E007E00703
:10923300E007E007E007E007E007E007E007E007F3
:10924300E007E007E007E007E007E007E007E007E3
:10925300E007E007E007E007E007E007E007E037A3
:10926300AC7672AD57AD38ADD8B5F9B5D9ADD9AD8A
:10927300D9ADD9ADD9ADD9ADF8ADF9ADD9AD983F2B
:109283008D07E007E007E007E007E007E007E007F6
:10929300E007E007E007E007E007E007E007E00793
:1092A300E007E007E007E007E007E007E007E00783
:1092B300E007E007E007E007E007E007E007E00773
:1092C300E007E007E007E0476D8E14AD37AD77ADFB
:1092D300D8B5F9ADD9ADD9ADD9ADD9ADF8ADF9B5ED
:1092E30099963507E007E007E007E007E007E007A6
:1092F300E007E007E007E007E007E007E007E00733
:10930300E007E007E007E007E007E007E007E00722
:10931300E007E007E007E007E007E007E007E00712
:10932300E007E007E007E007E007E007E007E057B2
:109333004E9DD5AD37A598ADF9B5F9ADD9ADD9AD3C
:10934300F8ADF9B579673007E007E007E007E00714
:10935300E007E007E007E007E007E007E007E007D2
:10936300E007E007E007E007E007E007E007E007C2
:10937300E007E007E007E007E007E007E007E007B2
:10938300E007E007E007E007E007E007E007E007A2
:10939300E007E007E007E067119DB6AD38AD98AD93
:1093A300F8B5F9ADF8ADB8A5D707E007E007E007D2
:1093B300E007E007E007E007E007E007E007E00772
:1093C300E007E007E007E007E007E007E007E00762
:1093D300E007E007E007E007E007E007E007E00752
:1093E300E007E007E007E007E007E007E007E00742
:1093F300E007E007E007E007E007E007E007E07EBB
:10940300B3A576AD38A5B8ADF8AD7876B207E00769
:10941300E007E007E007E007E007E007E007E00711
:10942300E007E007E007E007E007E007E007E00701
:10943300E007E007E007E007E007E007E007E007F1
:10944300E007E007E007E007E007E007E007E007E1
:10945300E007E007E007E007E007E007E007E007D1
:10946300E007E007E037AB7692A577AD37AD773706
:109473008C07E007E007E007E007E007E007E00705
:10948300E007E007E007E007E007E007E007E007A1
:10949300E007E007E007E007E007E007E007E00791
:1094A300E007E007E007E007E007E007E007E00781
:1094B300E007E007E007E007E007E007E007E00771
:1094C300E007E007E007E007E007E007E03FAC7EE6
:1094D30092671007E007E007E007E007E007E0070F
:1094E300E007E007E007E007E007E007E007E00741
:1094F300E007E007E007E007E007E007E007E00731
:10950300E007E007E007E007E007E007E007E00720
:10951300E007E007E007E007E007E007E007E00710
:10976300E007E0FFDFFFDFFFDFFFDFFFDFFFDFFFFC
:10977300DFFFDFFFDFFFDFFFDFF7BEFFDFFFDFFF1F
:10978300DFFFDFFFDFFFDFFFDFFFDFFFDFFFDFFFE6
:10979300DFFFDFFFDFFFDFFFDFFFDFFFDFFFDFFFD6
:1097A300DFFFDFFFDFFFDFFFDFFFDFFFDFFFDFFFC6
:1097B300DFFFDFFFDFFFDFFFDFF7BEF7DFF7DFF7F7
:1097C300DFF7BEF7BFF7BEF7BFF7BFF7BEF7DFF7A9
:1097D300BEFFDFFFBEFFDFFFDFFFDFFFDFFFDFFFD8
:1097E300DFFFDFFFDFFFDFFFDFFFDFFFDFFFDFF78E
:1097F300BEF7BEF7BEF7BEF7BEF7BEF7BFF7BEF7BD
:10980300BEF7BEFFDFF7BEFFDFFFDFFFDFFFDFFFD8
:10981300DFFFDFFFDFFFDFFFDFFFDFFFDFFFDFFF55
:10982300DFFFDFFFDFF7BEFFDFFFDFFFDFFFDFFF6E
:10983300DFFFDFFFDFFFDFF7BEFFDFFFDFFFDFFF5E
:10984300DFFFDFFFDFFFDFFFDFFFDFFFDFFFDFFF25
:10985300DFFFDFFFDFFFDFFFDFFFDFFFDFFFDFFF15
:10986300DFFFDFFFDFFFDFFFDFFFDFFFDFFFDFFF05
:10987300DFF7BEFFDFFFDFFFDFFFDFFFDFFFDFFF1E
:10988300DFFFDFFFDFFFDFFFDFFFDFFFDFFFDFF7ED
:10989300BEFFDFFFDFFFDFF7DFF7DFF7DEF7DFF71F
:1098A300BEF7DFFFDFFFDFFFDFFFDFFFFFFFFFFFAE
:1098B300FFFFFFFFFFFFFFFFFFFFFFFFFFFFFFFFB5
:1098C300FFFFFFFFDFF7DFF7DEEFDEEFBEE7BEE709
:1098D300BEE7BEE7BFEFDEF7DFFFFFFFFFFFFFFFE0
:1098E300FFFFFFFFFFFFFFFFFFFFFFFFFFFFFFFF85
:1098F300FFFFFFFFFFFFFFFFFFFFDFFFDFFFDFFFD5
:10990300DFF7DFF7BEF7DFF7BEFFDFFFDFFFDFFFC6
:10991300DFFFDFFFDFFFDFFFDFFFDFFFDFF7BEFF7D
:10992300DFFFDFFFDFFFFFFFDFFFDFFFDFFFDFFF24
:10993300DFFFDFFFDFFFDFFFDFFFDFFFDFFFDFFF34
:10994300DFFFDFFFDFFFDFF7BEFFDFFFDFFFDFF755
:10995300BEFFDFFFDFFFDFFFDFFFDFFFDFFFDFFF35
:10996300DFFFDFFFDFFFDFFFDFFFDFFFDFFFDFFF04
:10997300DFFFDFFFDFFFDFFFDFFFDFFFDFF7BEF725
:10998300DFF7DFFFDFFFDFFFFFFFFFFFFFFFFFFF6C
:10999300FFFFFFFFFFF7DFDFBFCF7EC73EAEDD9EDA
:1099A3007C9E1B8DDB6D5964F85CB85C7754574C17
:1099B300363C172B95237523351B341B351AF412AC
:1099C300F51AD31B141AF4231423142B3433553BE5
:1099D3005543B64BB553B653F6649885198D598DD7
:1099E300BAAE1BBE7CC6FDE77EF7BEFFFFFFFFFFDF
:1099F300FFFFFFFFFFFFFFFFFFFFDFFFDFFFDFFFD4
:109A0300DFFFDFFFDFFFDFFFDFFFDFFFDFFFDFFF63
:109A1300DFFFDFFFDFFFDFF7BEFFDFFFDFFFDFFF7C
:109A2300DFFFDFFFDFFFDFFFDFFFDFFFDFFFDFFF43
:109A3300DFFFDFFFDFFFDFF7BEFFDFFFDFFFDFFF5C
:109A4300DFFFDFFFDFFFDFFFDFFFDFFFDFF7BEFF4C
:109A5300DFFFDFF7BEFFDFFFDFFFDFF7BEFFDFFF65
:109A6300DFF7DFF7DFF7BFF7BFFFBFFFDFFFFFFF63
:109A7300FFFFFFFFFFF7DFD79EC73DA6BC8E9C65A8
:109A8300FA65BA45792CD814570BD603B603550398
:109A93005502D4031502F402F402B4029302D40271
:109AA3007302D4027302B402730253025301F2022B
:109AB3001201B1021201F202530A7312931AB41A79
:109AC300F42375335543754B7553954BB543954304
:109AD30095439543B53BD643B753B66CB864B86D5D
:109AE300398E3BAE9CC71DDF5EEFBFFFBEFFDFFFBE
:109AF300DFFFDFFFDFFFDFFFDFFFDFFFDFFFDFFF73
:109B0300DFFFDFFFDFFFDFF7BEFFDFFFDFFFDFFF8B
:109B1300DFFFDFFFDFFFDFFFDFFFDFFFDFFFDFFF52
:109B2300DFFFDFFFDFFFDFFFDFFFDFFFDFFFDFFF42
:109B3300DFFFDFFFDFFFDFFFDFFFDFFFDFFFDFFF32
:109B4300DFFFDFFFDFFFDFFFDFFFDFF7DFF7DFFF32
:109B5300DFFFDFFFFFFFFFFFFFFFFFDF9EB71D8E6E
:109B63009C5DDA45993D592D39457A3D79359A24DD
:109B7300F80CF90457041703F603D603F703950407
:109B830017039503B60375037503950375037502F0
:109B9300D40315029302D40AF413552BD65C576CE5
:109BA300F98DBA9E3CBEBDD71EE7BFEFDFF7DFFFDF
:109BB300FFFFFFFFFFFFFFFFFFFFFFFFFFFFFFFFB2
:109BC300FFFFFFFFFFFFFFF7DFEF7EE75ECEFDBE88
:109BD3009CAEBC965B9E9C965BA6BCBEBCDF3EF770
:109BE300BEFFDFFFDFFFDFFFDFFFDFFFDFFFDFFFA3
:109BF300DFFFDFFFDFFFDFFFDFFFDFFFDFFFDFFF72
:109C0300DFFFDFFFDFFFDFFFDFFFDFFFDFFFDFFF61
:109C1300DFFFDFFFDFFFDFFFDFFFDFFFDFFFDFFF51
:109C2300DFFFDFFFDFFFDFFFDFFFDFFFDFFFDFFF41
:109C3300DFF7BEF7BEF7DFF7DFFFFFFFFFFFFFFF33
:109C4300FFEFDFB71D865C5DDB35191D3A3519550E
:109C5300DB7E5C9EFDCF7EEFBEEFFF6E5B2D1904B6
:109C630017041703D6041704370416043703D6045E
:109C73001703B603F603B50376035502D403761B25
:109C8300B644B96D799E5BC71DE7BEFFFFFFFFFFBB
:109C9300FFFFFFFFFFFFFFFFFFFFDFFFDFFFDFFF31
:109CA300BEFFBFFFBFF7BFF7BEF7BEF7BFF7BEF7F5
:109CB300BFFFDFFFDFFFDFFFDFFFDFFFFFFFFFFF91
:109CC300FFFFFFFFFFFFFFFFFFF7DFF7BEF7BEF763
:109CD300BFFFDFFFDEFFDFFFDFFFDFFFDFFFDFFFB2
:109CE300DFFFDFFFDFFFDFF7BEFFDFFFDFFFDFFFAA
:109CF300DFFFDFFFDFFFDFFFDFFFDFFFDFFFDFFF71
:109D0300DFFFDFFFDFFFDFFFDFFFDFFFDFFFDFFF60
:109D1300DFFFDFFFDFFFDFFFDFFFDFFFDFFFDFFF50
:109D2300DFFFDFFFDFFFFFFFFFE7BFB6FD765B3D32
:109D330079151925193D7A7E3CB6FDDF9EF7DFFFC5
:109D4300FFFFFFFFFFFFFFFFDFFFDFF7DFEFBEC711
:109D53005D8E9C457A24B8043703D603F703D604F3
:109D630057039603B603B61C3745198DFBC73EEF61
:109D7300BEFFFFFFFFFFFFFFFFFFDFFFDFF7BEF7C2
:109D8300BFF7BEF7DFF7BFFFDFFFDFFFDFFFDFF761
:109D9300BEFFDFFFDFFFDFFFDFFFDFFFDFFFDFFFF1
:109DA300DFFFDFFFDFFFDFFFDFF7BFFFDFFFDFF7F0
:109DB300BFF7BFF7BEF7DFFFDFFFDFFFDFFFDFFF29
:109DC300DFFFDFFFDFFFDFFFDFFFDFFFDFF7BEFFC9
:109DD300DFFFDFFFDFFFDFFFDFFFDFFFDFFFDFFF90
:109DE300DFFFDFFFDFFFDFFFDFFFDFFFDFFFDFFF80
:109DF300DFFFDFFFDFFFDFF7DFFFDFFFDFFFDFFF78
:109E0300DFF7DEFFDFFFDFFFDFFFBEFFDFFFDFFF89
:109E1300DFFFDFD79E7EDC3DBA25191CB83D9A7E55
:109E23005BBF3DEFBFFFFFFFFFFFFFFFDFF7BEF7A6
:109E3300BFF7DFF7DFF7BEFFDFFFDFFFDFFFDFFF88
:109E4300FFFFFFFFFFE7BEC73D8E5B4D5A1C770C3C
:109E530058247875DBB6FDE79EFFFFFFFFFFFFFF8A
:109E6300DFF7BEF7BEF7DFFFDFF7DFFFDFFFDFFF61
:109E7300DFFFDFFFDFF7BEFFDFFFDFFFDFFFDFFF18
:109E8300DFFFDFFFDFFFDFFFDFFFDFFFDFFFDFFFDF
:109E9300DFF7BEFFDFFFDFFFDFF7BEFFDFFFDFFF21
:109EA300DFFFDFFFDFFFDFFFDFFFDFFFBFFFBFFFFF
:109EB300DFFFDFFFDFFFDFFFDFFFDFFFDFF7BEFFD8
:109EC300DFFFDFFFDFFFDFFFDFFFDFFFDFFFDFFF9F
:109ED300DFFFDFFFDFFFDFFFDFFFDFFFDFFFDFFF8F
:109EE300DFFFDFF7DFF7DFFFDFFFDFF7BEF7BEF7E9
:109EF300BEF7BEF7BEF7BEFFDFFFDFFFDFF7BEF73C
:109F0300BEFFBEC73D8EDC96BCBF1DE7BEFFFFFF95
:109F1300FFFFFFFFBEFFBEF7BEF7BFFFDFF7DFFFA9
:109F2300DFFFFFFFDFFFDFF7BEFFBEFFDFF7DFF778
:109F3300BEF7BEF7BEFFBEFFDFFFFFFFFFE79ECF0B
:109F43005DF7FFFFFFFFFFFFDFF7BEF7DFF7BEF7AA
:109F5300BEF7BEF7BEF7BEFFDFF7BEF7BEF7BEF72D
:109F6300BEF7BEF7BEF7BEF7BEF7BEFFDFFFDFF7F4
:109F7300BEF7BEF7BEF7BEF7BEF7BEF7BEF7BEF736
:109F8300BEF7BEF7BEF7BEF7BEFFDFFFDFFFDFFFA3
:109F9300DFFFDFF7BEF7BEF7BEFFDFF7BEFFDFFF72
:109FA300DFFFFFFFFFFFDFFFDFFFDFFFDFFFDFFF7E
:109FB300DFF7BEF7BEF7BEF7BEF7BEF7BEF7BEFFCD
:109FC300DFF7BEFFDFF7BEF7BEF7BEFFDFFFDFFF42
:109FD300DFFFDFFFDFFFDFFFDFFFDFFFFFFFFFFF4E
:109FE300FFFFFFFFFFFFFFFFDFF7BEF7BEFFFFFF30
:109FF300FFFFFFFFFFFFFFFFFFFFFFFFFFF7BEF7BF
:10A00300DFF7FFFFFFFFFFFFFFFFFFFFFFFFDFFFA5
:10A01300BEFFBEFF9EFFDFFFFFFFFFFFDFFFFFFF70
:10A02300FFFFFFFFFFFFFFFFFFF7DFF7DFFFFFFF8D
:10A03300FFFFDFF7DFFFFFFFFFFFFFFFDFFFFFFF95
:10A04300FFFFFFFFFFFFFFFFFFFFFFFFFFFFFFFF1D
:10A05300FFFFFFFFFFFFFFFFFFFFFFFFDFFFFFFF2D
:10A06300FFFFFFFFFFFFFFFFFFFFFFFFFFFFFFFFFD
:10A07300FFFFFFFFFFFFFFFFFFFFDFFFDFFFDFF755
:10A08300BEFFFFFFFFFFFFFFFFFFFFFFFFFFFFF726
:10A09300BEF79EF79EF7BEFFDFFFFFFFFFFFDFFF69
:10A0A300DFFFFFFFFFFFFFFFFFFFFFFFFFFFFFFFDD
:10A0B300FFFFFFFFFFFFFFFFFFFFFFFFDFFFDFFFED
:10A0C300DFFFDFFFDFFFDFF7BEFFDF8430630C63FB
:10A0D3002C632C738EAD55F79EFFFFFFFFD69A843A
:10A0E30010630C630C5B0C634DDEFBFFDFFFFFFFB4
:10A0F300FFFE59FCB2FB4DFACBF9C7F924F924F959
:10A10300A6FA08FA49FA69FA69FAEBFF1CE75D6BEC
:10A113006D630C630C630C9CF3FFFFFFDFFFDFFF3A
:10A12300DFFFDFFFFFAD75630C9CD3FFFFDEDB6357
:10A133002C630C630C630C5AEB528A4A694A6952CA
:10A143008A4A69528A528A528AB596FFDFEF5D6B5B
:10A153006D630C630C630C5AEB528A528A528A5217
:10A163008A528A5ACB8410B5B6FFDFFFDFFFDFFFC9
:10A17300FFE73CB5968410630C4A69318621242994
:10A183006542084A49528A528A528A9492FFDFFFF3
:10A19300FFBDF78C516B4D630C52AA4A694A494A79
:10A1A300494A494A69528A7BEFD69AFFFFFFDFFF8C
:10A1B300DFFFDFFFDFFFDFF7BEFFFF3186000000B9
:10A1C3000000000000000029658C515ACB000000FC
:10A1D300000000000000000000AD55FFFFF659F934
:10A1E300E7F841F800F800F800FAAAFD14FE59FE5A
:10A1F300BAFEFBFF1CFEBAFE59FE18FFBEBDF700F8
:10A203000000000000000031A6FFFFF7BEFFDFFFE4
:10A21300DFF7BEFFFF4A4900003186FFFFB5960016
:10A223000000000000000010A2AD55B5B6B5B6B5EC
:10A23300B6BDD7B5B6B5B6B5B6DEDBFFFFC61800FB
:10A243000000000000000010A29CD3A534A534A593
:10A2530034A5148C71210400006B6DFFFFFFDF7BBD
:10A26300EF18C300000000000010A28410BDD7D671
:10A27300BAEF7DF79EEF7DDEFBCE79D6BAFFFF7B8B
:10A28300CF00000000000000006B6DB596BDD7BD88
:10A29300D7B5B6B5B67BEF00000861D69AFFDFF7F6
:10A2A300BEFFDFFFDFFFDFF7BEFFFF4208000063F3
:10A2B3000C632C0841000000000000084184304278
:10A2C300080000002000200000B5B6FF7DF0E3F891
:10A2D30000F800F820F800FC51FFFFFFFFFFFFFF2D
:10A2E300FFFFFFFFFFFFFFFFFFF7FFFFFFBDF700CC
:10A2F300000020002000004208FFFFF7BEFFDFFF41
:10A30300DFF7BEFFFF528A00004208FFFFBDD70000
:10A313000000200020000018E394B29CF39CF39CFF
:10A32300F39CF39CF39CF3CE59FFFFFFFFC6380069
:10A33300000020002000004228FFFFFFFFFFFFFF77
:10A34300FFFFFFFFFF8C5100002945FFFF8C7100C9
:10A353000000000020002018E3E71CFFFFFFFFEFD1
:10A363007DD69AD69AD69ADEFBE73CFFDFFFFF3114
:10A37300A60000002000200000738E949294929413
:10A3830092949294927BCF00200000B5B6FFFFF722
:10A39300BEFFDFFFDFFFDFF7BEFFFF42080000ADB8
:10A3A30055FFFFCE7994926B6D94B2E71CFFFF5A71
:10A3B300EB0000000000000000B5F7FE9AF000F883
:10A3C30020F800F800F800FE79FFFFFF9EFFBEFFB4
:10A3D300BEFFBEFFBEFFBEFFBEF79EFFFFBDF70081
:10A3E300000020000000004208FFDFF79EF7BEF7E1
:10A3F300BEF79EFFDF528A000039E7FFFFBDD7009B
:10A403000000000000000000204A695ACB5ACB5AD2
:10A41300CB5ACB5ACB5ACB8410FFDFFFFFC6380091
:10A4230000000000000000084152AA632C630C6383
:10A433000C5AEB4A6908412965A534FFFF422800FD
:10A44300000020002000004228FFFFF79EF7BE8493
:10A453003039C739C73186086100004A69FFFF42B6
:10A463000800000000000000004208738E738E7322
:10A473008E738E738E4A4900000000BDF7FFFFFF05
:10A48300DFFFDFFFDFFFDFF7BEFFFF420800009CB7
:10A49300D3FFDFFFFFFFFFFFFFFFFFFFFFFFDF52E2
:10A4A3008A0000002000200000B575FFDFFA69F87C
:10A4B30000F800F800F800FA8AFF3CFFFFFFFFFFF7
:10A4C300FFFFFFFFFFFFFFFFFFF7FFFFFFBDF700EA
:10A4D300000000000000004208FFFFFFFFFFFFFF36
:10A4E300FFFFFFFFFF528A000039E7FFFFBDD700E0
:10A4F3000000000000000039C7FFFFFFFFFFFFFF60
:10A50300FFFFFFFFFFFFFFFFFFF7BEFFFFCE590077
:10A513000000000000000018E38C518C718C518CFA
:10A52300518C71A534CE79F79EFFFFFFFFBDF70075
:10A53300200000000000001082BDF7FFFFFFFFFFB7
:10A54300FFFFFFFFFFFFFF5ACB000039C7FFFF39B3
:10A55300E70000002000200000CE59FFFFFFFFFFAF
:10A56300FFFFFFFFFFD6BA00000000BDF7FFFFF7B4
:10A57300BEFFDFFFDFFFDFF7BEFFFF318600009C7A
:10A58300F3FFFFF7BEF7BEF7BEF7BEF7BEFFFF52FE
:10A59300AA0000000000000000B5B6FFFFF79EFC14
:10A5A30051F986F882F800F800F841FA28FBCFFC4D
:10A5B30092FC92FC92FC71FC51FC10FF1CEF7D633A
:10A5C3000C10A200200000000042085ACB5AEB5A9C
:10A5D300EB5AEB42280000000039E7FFFFEF7D73E1
:10A5E3008E21040841000031A6FFDFF7BEF7BEF756
:10A5F300BEF7BEF7BEF7BEF7BEFFDFFFDFF7BE73E2
:10A603008E18C30000000039E7FFFFFFFFFFFFFFC5
:10A61300FFFFFFFFFFFFFFFFDFF7BEFFDFFFFFC609
:10A62300385ACB18E30841000000004A698C719442
:10A63300B294B294928C511082000031A6FFFF397C
:10A64300C70000000000000000BDD7FFDFF79EF742
:10A65300BEF79EFFDFC63800000000BDD7FFFFFF37
:10A66300DFFFDFFFDFFFDFFFDFFFDFBDD7A534EF56
:10A673007DFFDFFFDFFFDFFFDFFFDFFFDFFFDFDE6A
:10A68300DB9CF39CF39CF3AD55F79EFFDFFFDFFFED
:10A69300FFFFDFFEBAFDD7FCF3FC51FB4DFAEBFAEB
:10A6A300EBFAEBFB0CFBAEFC30FCD3FF7DFFFFFFB3
:10A6B300FFDEFBC618A5349CF38C718C718C718CF6
:10A6C300718C718C719CF3A534D69AFFDFFFDFFF89
:10A6D300FFEF5DCE59AD75CE79FFDFFFDFFFDFFF03
:10A6E300DFFFDFFFDFFFDFFFDFFFDFFFDFFFDFFF77
:10A6F300FFE71CBDF79CF3D69AF7BEF7BEF7BEF78C
:10A70300BEF7BEFFDFF7BEFFDFFFDFFFDFFFDFFFC9
:10A71300FFFFFFEF5DC638AD559CD373AE630C5A94
:10A72300CB5ACB5AEB6B4D84309CD3CE59FFDFCE43
:10A7330079A5149CF39CF3AD75F79EFFDFFFDFFF54
:10A74300DFFFDFFFDFF7BEB596AD55EF7DFFDFFF20
:10A75300DFFFDFFFDFFFDFFFDFFFDFFFFFFFFFFFC6
:10A76300FFFFDFFFDFFFDFFFDFFFDFFFDFFFDFFFD6
:10A77300FFFFFFFFFFFFFFFFFFFFFFFFDFFFDFFF26
:10A78300BEFFDFFFFFFFFFFFFFFFFFFFFFFFFFFF37
:10A79300FFFFFFFFFFFFFFFFFFFFFFFFFFFFDFF7EE
:10A7A300BEFFFFFFFFFFFFFFFFFFFFFFFFFFFFFFF7
:10A7B300FFFFFFFFFFFFFFFFFFFFFFFFDFFFDFF7EE
:10A7C300BEFFFFFFFFFFFFFFFFFFDFFFDFFFDFFF37
:10A7D300DFFFDFFFDFFFDFFFFFFFDFFFDFFFDFF76E
:10A7E300BEFFFFFFFFFFFFFFFFFFDFFFDFFFDFFF17
:10A7F300DFFFFFFFFFFFDFFFDFFFDFFFDFFFDFFF26
:10A80300DFFFDFFFFFFFFFFFFFFFFFFFFFFFFFFF95
:10A81300FFFFFFFFFFFFFFFFFFFFFFFFFFFFDFFF65
:10A82300FFFFFFFFFFFFFFFFFFFFFFFFDFFFDFFF75
:10A83300DFFFDFFFDFFFDFFFFFFFFFFFFFFFDFFFC5
:10A84300DFFFDFFFDFFFDFFFDFFFDFF7BEF7BEFF67
:10A85300DFFFDFFFDFFFDFFFDFFFDFFFDFFFDFFF05
:10A86300DFF7BEF7BEF7BEF7BEFFDFFFDFFFDFFF99
:10A87300DFFFDFFFDFFFBEFFBEFFBEFFBEFFBEFF8A
:10A88300BEFFBEFFBEFFBEFFBEFFBEFFDFFFDFFF9B
:10A89300DFFFDFF7BEF7BEF7BEF7BEF7BEF7BEF7C3
:10A8A300BEF7BEF7BEF7BEF7BEFFDFFFDFFFDFFF7A
:10A8B300DFFFDFFFDFF7BEF7BEFFDFFFDFFFDFFFF7
:10A8C300DFFFDFFFDFFFDFFFDFFFDFFFDFFFDFFF95
:10A8D300DFFFDFFFDFF7BEF7BEFFDFFFDFFFDFFFD7
:10A8E300DFFFDFFFDFFFDFFFDFFFDFFFDFFFDFFF75
:10A8F300DFFFDFFFDFFFDFF7BEF7BEF7BEF7BEF711
:10A90300BEFFDFF7BEF7BEF7BEF7BEFFDFFFDFFF19
:10A91300DFF7BEF7BEF7BEF7BEFFDFFFDFFFDFFFE8
:10A92300DFFFDFFFDFFFDFF7BEF7BEFFDFFFDFFF86
:10A93300DFFFDFFFDFFFDFFFDFFFDFFFDFFFDFFF24
:10A94300DFFFDFFFDFFFDFFFDFFFDFFFDFFFDFFF14
:10A95300DFFFDFFFDFFFDFFFDFFFDFFFDFFFDFFF04
:10A96300DFFFDFFFDFFFDFFFDFFFDFFFDFFFDFFFF4
:10A97300DFFFFFFFDFFFDFFFDFFFDFFFDFFFDFFFC4
:10A98300DFFFDFFFDFFFDFFFDFFFDFFFDFFFDFFFD4
:10A99300DFFFDFFFDFFFDFFFDFFFDFFFDFFFDFFFC4
:10A9A300DFFFDFFFDFFFDFFFFFFFDFFFDFFFDFFF94
:10A9B300DFFFDFFFDFFFDFFFDFFFDFFFDFFFDFFFA4
:10A9C300DFFFDFFFDFFFDFFFDFFFDFFFDFFFDFFF94
:10A9D300DFFFDFFFDFFFDFFFDFFFDFFFDFFFDFFF84
:10A9E300DFFFDFFFDFFFDFFFDFFFFFFFDFFFDFFF54
:10A9F300DFFFDFFFDFFFDFFFDFFFDFFFDFFFDFFF64
:10AA0300DFFFDFFFDFFFDFFFDFFFDFFFDFFFDFFF53
:10AA1300DFFFDFFFDFFFDFFFDFFFDFFFDFFFDFFF43
:10AA2300FFFFDFBD59A474E679E697D5D2EE95E62C
:10AA330035E5F5EE57FED8EE75EE74FF17F6D7AC95
:10AA4300D1A470B4F2B512A4B0942EACD1A470A466
:10AA530091A4719C91A492ACD3A4B3A493A4B3ACDA
:10AA6300F5A4B4A4B5A4D6ACF69C94949394D48CD6
:10AA7300928C937C527C737433849684D88CD9746F
:10AA8300379D5B95178CD595168CF58CD5951694BB
:10AA9300D68CB594B69CF79CB79CD7ACB7CD99D65A
:10AAA300176AA76265EE95DDF46A268B2AE5F5EE53
:10AAB30034B4CEC530E6969C0E49A5ACB0BD526AFF
:10AAC300C949C583ADB5137B4C5A286AEB9430BD95
:10AAD30076BD75BD55ACF4B515B515BD57ACF6A42B
:10AAE300B49CD48C3173CF843184717411743284E7
:10AAF300B4745484B77C768CD9953A849574127C5B
:10AB030073741273D16BD17BF37C33A538AD59A524
:10AB130018AD39ACD8B4F6E679CDB3C571FEF6D528
:10AB2300928B2A9BCCE635EE75C550CD71EE96AC73
:10AB33009072C99C2FC573940E6AC97B6C9C707B01
:10AB43004B6ACA838D8BCE8BCF7B6D8C109C519CB3
:10AB5300718BF09431943294517BAE83EF84506BBC
:10AB63006D73EE73EF74107C9384D58D177C7584AD
:10AB7300B87C9684954ACD42AC4AED5B2F428C4A11
:10AB83006D52EE8C559CF794969CB6C57AACB6DEA6
:10AB930038E697DE34F6B5F696FEB8EE36F676EE80
:10ABA30054EE74EE95E675BD12BD53B512B512B5EC
:10ABB300328BCD940EACF1ACF283AD942FACF2BDDD
:10ABC30074B5549450B534CDD6C5D6A492A4D373DA
:10ABD3004C6B2BA512B594AD94CEB8A5948CD25BD7
:10ABE3006D7C7284D584B57C969D7963D1532E4A4E
:10ABF300ED42AC4AAD63705AEF4A6D8414AD79AD42
:10AC030059AD39ACB7B4D6DE58E697E654FEF6F63E
:10AC130096E615F677EE56EE54F6B5F6D6E696BDFD
:10AC230012BD33BD53A4B09C4F72EA940EC5B4C594
:10AC33009483ADACF1C5D5CE16CDF66B0A9470AD49
:10AC430012ACF2E6B9CE1683CDB553C615948EB5C4
:10AC5300B3C656E75ACED984907C518CF484B46B36
:10AC6300F295583A4B3A4B3A6C530E3A4C52EE42E9
:10AC73006C52EF52AE94969CD79496C57ABD17DE6C
:10AC830038F719F6D6EE95EE56F697F657F677F6A9
:10AC930095F6D6F6D6EED7BD32A491B533A4907B04
:10ACA3006B838CB512CDD5942EA490CE15C5B494D8
:10ACB3004E944E6B0ABDB4BDB4A4F1A4B07B8BBD5E
:10ACC30073CE35AD30B572BDB3BDF3AD93C656B5D6
:10ACD300F57C50955595358CD5A5B94ACD3A6B423F
:10ACE3008C63904ACE530F4A6D5B3063309CF7B54B
:10ACF30079AD38ACB7B4F7DE58EED8EE95EE74EE16
:10AD030056F677F697F676F675F6D6EEB5EE96BD69
:10AD130012A470BD538BCD6AEAACF1EED9CDD573D5
:10AD23004BB512E6B8E6D8A4D08C2D9CAFD676B539
:10AD330072948E8C0D83CCEF19A4CF7349C5F3ADF8
:10AD430030A530AD92BE35CED97C506BF07C737C90
:10AD5300738D16534F532F530E322B426C639163F3
:10AD6300303A2C739294969CD79CD7BD19BD58D674
:10AD730017E697EE95F6B5F696F657EE57F697FE65
:10AD8300B6FEF6EEB5EEB6BD129C50A4706AC98B42
:10AD9300CDB512D6369C8F7B8BBD73D635DEB7947B
:10ADA3004D62E8B592DE96A510944D6AE8B532C5BA
:10ADB300B383AB62E783CB7B8A5AC7840C8C6FBEA9
:10ADC300169D1363AF953684B4953784B54ACE5335
:10ADD3000F4ACE6B914ACE635073D39CF8A538A526
:10ADE30019AD59ACD8B4F7DE58F6F8F6D6F6B5F681
:10ADF30076FE98F697F697F6B6F6B5EEB5F6D7B4AF
:10AE0300F1A470940E5A885A47B553DE978BCD6AD6
:10AE1300E9C5D4E6F8D6557BCB4A246B49C613B5AE
:10AE2300927BAA5246CDD5DE97ACF0734983CB7B98
:10AE33008A5AA752875AE98C71ADB66BD07C538C72
:10AE4300F684B66BF3530F42AE4ACE5B304ACE4A1A
:10AE53008E73B2841494B6A518A4F8ACD8B4F7DEF4
:10AE630038EED8EEB6F6B5EE76F697F697F677F6B1
:10AE7300B6F6B5EEB5F6D7B512A490942F52267B4D
:10AE83008C9C6FCDF58BED5226AD51DED7CE357B45
:10AE9300AB62E79CAEB591E6F7A4EF5A8783ACCDDE
:10AEA300F5E6B8B531B531B5318C2D5AC85AEA8CAF
:10AEB30051A555638F8CF6849584B66BD25B715B19
:10AEC300504ACE52CE530F5B1073B27BD39496A4E9
:10AED300F89CD8B4F8B517DE38EED7EEB5F6B5EE74
:10AEE30076F697F697F677F6B6F6B5EE95F6D7B407
:10AEF300F1A4908BCD8BED83CD8C0EC5B4AD118CAD
:10AF03000D840CB551E6D7AD519CAE73AAA530DEC6
:10AF1300D6BDB3946F83CDA4D0C5D4E6D8CE15A443
:10AF2300AFA4D0840E73ADA5559D1574129D5874AE
:10AF33005574344B0F533063B2533052EF6BB26BD3
:10AF4300714A8E63318435A4F8A518B518BD17DE90
:10AF530058EED8EEB6F6B5F676FE98FE98F697F666
:10AF6300B6F6B5EE95EEB7B4D19C4F7B4BBD53838C
:10AF7300CCACF1C5D4C5D4B5527BABD656E6F7B548
:10AF830092AD307BCBDEB7CE349CCFA5116B2AAD0F
:10AF930032D636E6B7DE97B57283ED83EE73ADAD89
:10AFA3007573F0849484D67C9563D34AEF530F630F
:10AFB300924AAE320C635173D35AF0528E73929C01
:10AFC300B7A518B519BD17DE38EED8EEB6F6B5F647
:10AFD30076FE98F697F697FEB6F6B5EEB5EEB6ACF6
:10AFE300B09C2F7B4B9C8F946FBDB4BDB4A4F08CED
:10AFF3002E8C2DDED8AD51840C83EB9CAECE35B5B3
:10B00300B373AB8C2D738BC5F4CE35C5F4CDF4B5CA
:10B0130072944E949094B1A555634E849474337C8A
:10B023009663D363926BD284966BB3426E637284DE
:10B03300557BF46B518435A518AD59B4F8BD17DEB3
:10B0430038EED7EEB6F6B5F676F697F677F677F6E8
:10B05300B6F6B5EEB5EED7B4D19C2F734B8C0D9CE1
:10B063008FAD11CE358C2D9C8F8C0DCE35D676942D
:10B073008F9CCF9CD0BDD3D6979CD08C2D94AFBD45
:10B08300D3BDB3CE14C5D3AD11B572B593C616A552
:10B09300556BAF7C937C9484F784D67C756BD38497
:10B0A300767C556B927C1484356B9284148C769CDD
:10B0B300D79CD7B4F8B517DE38EED8F6D6F6D6F661
:10B0C30076F697F677F677F6B6F6B5EEB5F6D7B425
:10B0D300F1A47083AC8BED9C8F9C6FD656A4D0B536
:10B0E30072946EAD32DED8A4D0A4F08C4EBDD4CE13
:10B0F300769CF094AF842CAD71DEB6D655DED6DEE9
:10B10300D7BDB3AD52B5B49D335B4D84B38D368596
:10B11300169DBA8D1863B25B51531052F06BB37323
:10B12300D36B72A539AD59AD39AD39B4F8B517DE66
:10B1330038EED8F6F7F6F7F696F6B7F6B8F697F6CA
:10B14300B6EE96EEB6F6D7BD12ACB09C6F6B09B5F2
:10B15300729C8FBD93BDB38C4EBDB39CAFB572C50E
:10B16300F49CD0A4F0A4F0B572AD7294AFA5309462
:10B17300AEAD30B591CE34CE14CE35BDF5B5D5B523
:10B18300F7532C8D158CF56C5385178CD774147C61
:10B19300346BB35B316B927C148C76949694969457
:10B1A300979CB7BD38B4D6DE59E678DE56E675F619
:10B1B300F8F6D7E676EEB7FF39EE97F6D8EEB7BDD9
:10B1C30032A48F9C8F63099CD0948F6309A5118C43
:10B1D3002DAD318C4E83ECBDD3944EA4F06B4984DA
:10B1E3000CA4F083EC9CAE7369944DA4CFC5F4C654
:10B1F30035CE77CE78B5F6BE386BAF741184D5955E
:10B20300378D179538951895188CB78C969D18A57A
:10B2130039B59AA518A4F8B57AB559B4D6BD16EEC2
:10B223009BBD3462A8940CE696EEB6F718EEB7AC65
:10B23300D0ACB08B8BD5D4BD11ACAFAD11736B4A11
:10B24300465266736BAD32C5D48C2D5246A510CED3
:10B2530055A4F083EC4A25946ECE35ACF052457B71
:10B263008AA4CFBDD3B573CE77B5D5C6378C9184B9
:10B273009273F0951584B47C747C54741374137CAA
:10B283003473F373F3843473B26B517BB37B929453
:10B29300559CB6B4B5B4B4E65AD5F6940DB4F0E6FD
:10B2A30096E655EE96DE148B8BAC6F7B09DE15C5E7
:10B2B300529C4EA4B09CB0736B8C2EA4F1B552DE9D
:10B2C30098B573B552A4D0AD31E6B8C5D4A4AFB523
:10B2D30052B531CE35A4CF946E9C8FA4F0B5939C18
:10B2E300B09D127BEE73CE73EF52EC5B4E6BB08C62
:10B2F300B495167C548D179D38741373F39CF7A57E
:10B30300189CB69CD79455A4D7AD39CD78C536CD06
:10B3130097A4709C2D9C0CC571EED6EE96E656A4B0
:10B323004EAC8F9BEDC552C552AC8FBD738C2E7343
:10B333004BC5B4D657D636A4D1AD12DE77B532BDE0
:10B3430093B5539C6FBD93BD73A4B09C6FA4D0D62B
:10B3530056AD11946E8C4E8C4F5AE95AEA3A07292E
:10B36300A63208424A29C83A4A4AAD639074548CBB
:10B37300D68475845494D6843473929CB68C35A445
:10B38300B7AD18AC95BD36EE9BCDB6EEB8D614E688
:10B3930096EED7E696F6F8CD93CD73CD93C552BD11
:10B3A30011BD11ACF183CD944FCDF6AD128BEE6A86
:10B3B300EAC5B4C5D5B5338BCD62A9A4D1CDF69C6E
:10B3C3007083CD736BB553C5F5AD32736B422642B3
:10B3D3000539C53A0652A94A693A08298631C83A55
:10B3E3002A3209322A196729C9530E845494B57B2A
:10B3F300F37BD37BB27BB29C96A4F8BD17ACB5E6C6
:10B403007AE658E677ACCFACAF942CA48EBD119CF2
:10B413000DC552EEB8EE97B4D0ACD0ACF2942F94E5
:10B423002FA4B19C70732B734CACF29C70A4B17BB2
:10B433008D7BADB5339C90945083CD736CCE168CBD
:10B443000E7BCD52884A674A4794906B6C3A072922
:10B45300645AEB5AEC4A8B3A095B0D7432532E3A19
:10B463004B31EA5B0E8C959CD69CD6A4D79CB6B583
:10B4730039B539B517ACD6D619E69ACDD59C4E94C5
:10B483002DACD09C8E9C4E8BACACB1D616E6B8B529
:10B4930012B4F1AD12A4D19CB19CB19C919450947F
:10B4A300709CB1A4F2AD13A4D294719471A4F3C5AA
:10B4B300F78C509C919CB19CD26B4C528842277B59
:10B4C300EE8C4F738D6B4C6B6D845073AE7BEF4A78
:10B4D3006A52CC5B6F5B8F4AED29C9426C8C749CBA
:10B4E300F794B69CD79455A4B7A4F8ACF8ACF77B03
:10B4F30090732D8BEE9CB0736B8C2D83ED8BED9C39
:10B50300908BCE83AD7B6C62A962C96B0A62EA6BD6
:10B513002B630A4A27738C528962EB6B2B52A96BFC
:10B523004C738D6B6D6B6D5AEB738D738D6B2C73CD
:10B533006D5AEA52895289632B9D128C505AEA4202
:10B54300275B0B6B6E94B3528A424A5B4E3A8B3243
:10B553000929E94A8C6B706B70737162EF5AAF8380
:10B56300F4AD189CB79CB76B4F62CC632B52A95AAE
:10B57300C96B2A630A5A886B2B5A8952284A075A7D
:10B583006852474A274A4742274A684A884A684ACC
:10B5930068420739E739E742485AEB5B0C4AAA4A43
:10B5A3006A52AA630C526931A639E75ACA52AA529F
:10B5B300CA7BCE73AD422842284A694A694A6A4225
:10B5C3002952EC5B4E4B0D4ACC428C424B3A0A4219
:10B5D3000B422C5ACF526D7B92A4D8B57AAD397BEE
:10B5E300B1630D630C4A68422642475288420652B1
:10B5F3008942084A2852695ACA5AC94A474A684A74
:10B603006852A952C952A94A89422842083A0842B3
:10B61300695AEC5B0C52CB4AAB52CC6B6E62EC4A70
:10B623002939E84A494A4942284A895B0B4AAA4AC6
:10B63300AA3A2831E8426A424A426A3A4B322A32EB
:10B643002A320A3A0A39EA39EA420B5AAF5A8E8346
:10B65300D4B5399CD894966B2F5AAC5ACB4A684AC6
:10B66300474A6752A94A2752894A4852695AAA5AED
:10B67300A9526852A852885288528852A952A95294
:10B68300894A694A4942494A8A5AEC52EC52AB4ABE
:10B69300AB52CC52AC528B4A4A39E842294A8A4AC5
:10B6A3008A424942694A8A4AAB3A0831E8426A42C5
:10B6B3006A426B3A4B324B322B3A4B3A2C3A0B429F
:10B6C3000B420C4A2D4A2D7372A4B8AD39B559A457
:10B6D300F6AD15B595B594B573BDB4BDB4B553BD4D
:10B6E30095B574B575B5549C918C0E9C908C2E8C2D
:10B6F3000E83CD83EE8C2F8C2F8C51843084318C30
:10B70300518C728C528431843284528C528C538C7F
:10B71300327BF173D07C317C106BAE636D5B4D6318
:10B723006E63AF6BAF638F63B07C537C747C747C4C
:10B73300547C54845484148414841483D37BB3942A
:10B7430056AD19ACD7B558CE1ADE9AEEFAE6D9DE65
:10B7530097DEB7DEB7DE97E698E699E6B9E698BDD9
:10B7630053A4B1B5129C6F9C70940F942F9C719C41
:10B7730051A4D39CB2A4B3A4B39CB49C9394939CC0
:10B78300949CB49CD59CD59CD59CD48C738C73848D
:10B79300727C117C527C31743184D4953684B484A8
:10B7A300D49D988CD684B68CB68CB694B794B79C3B
:10B7B300D7A4F8A4D79CB7A4B8A4F8B4F7BD37D6D8
:10B7C3003ADE9ADE98DE97DE56E696DE76DE77DEA2
:10B7D30057DE57E678E677BD32ACD1BD12A46FAC25
:10B7E300B1A470A491ACB29C50A4B3A4B3ACD4AC38
:10B7F300F4A4D4A4B4A4B4ACF5AD16949494B49CBA
:10B80300D59CF59CD58CB48C938CB37C3284937487
:10B81300327C7384F57C947CB48D168D178CD78C15
:10B82300D78CD794D79CD89CF8A519A4F9AD19AD9A
:10B8330019AD192000000000000000000000000006
:10B84300000000002200000000000014282850001F
:10B8530000000000002C0000000000001818083051
:10B863000000000000002D0000000000000000FEAA
:10B87300000000000000002E00000000000000187F
:10B8830018000000000000003000000018244242AD
:10B8930042424242241800000031000000107010A0
:10B8A3001010101010107C000000320000003C4209
:10B8B300420204081020427E000000330000003CD6
:10B8C30042420418040242423C00000034000000DB
:10B8D3000808182848487E08081E000000350000A4
:10B8E300007E40405C62020242423C00000036009F
:10B8F30000001C2440405C624242423C000000378E
:10B903000000007E444408081010101010000000CE
:10B91300380000003C4242423C244242423C000088
:10B92300003900000038444242463A0202243800FB
:10B9330000003A000000000018180000001818006A
:10B943000000003B000000000800000000000808A1
:10B9530010000000410000001010282828287C4413
:10B9630044EE00000042000000FC4242447844429E
:10B973004242FC000000430000003E42828080807F
:10B983008082443800000044000000F844424242F0
:10B9930042424244F800000045000000FC4248488F
:10B9A3007848484042FC00000046000000FC424842
:10B9B300487848484040E0000000470000003C440D
:10B9C300848080808E84443800000048000000EEAC
:10B9D3004444447C44444444EE00000049000000D5
:10B9E3007C10101010101010107C0000004A000092
:10B9F3003E08080808080808080888F000004B00FB
:10BA03000000EE4448507050484844EE0000004C9B
:10BA1300000000E04040404040404042FE00000043
:10BA23004D000000EE6C6C6C5454545454D600001A
:10BA3300004E000000EE64645454544C4C4CE4003B
:10BA430000004F00000038448282828282824438A0
:10BA530000000050000000FC4242427C4040404055
:10BA6300E00000005100000038448282828282B2EA
:10BA73004C3806000052000000F844444478504813
:10BA83004844E6000000530000003E424240300CB0
:10BA93000242427C00000054000000FE921010108D
:10BAA300101010103800000055000000EE4444440C
:10BAB30044444444443800000056000000EE44442B
:10BAC3004428282828101000000057000000D654EE
:10BAD3005454546C2828282800000058000000EE15
:10BAE3004428281010282844EE00000059000000C4
:10BAF300EE4444282810101010380000005A0000AB
:10BB0300003E44040808101020227E0000005B0061
:10BB1300003C20202020202020202020203C00004A
:10BB23000040402020101010080804040402005DA7
:10BB330000003C04040404040404040404043C005E
:10BB43005E00000000000000182400000000000058
:10BB5300005F0000000000000000FE000000000085
:10BB6300000060000000000000003008000000003A
:10BB730000000061000000000038441C2444443EDF
:10BB83000000000062000000C040405C624242428C
:10BB9300427C0000006300000000001C2240404083
:10BBA300221C00000000640000000C04047C848458
:10BBB30084848C760000006500000000003C427E17
:10BBC3004040423C00000000660000000E12107C62
:10BBD30010101010107C00000067000000003E44AD
:10BBE3004438403C42423C00000068000000C04032
:10BBF300405C6242424242E70000006900000030BC
:10BC030030007010101010107C0000006A00000C4F
:10BC13000C001C040404040404447800006B0000BA
:10BC230000C040404E4850684844EE0000006C009D
:10BC330000007010101010101010107C0000006D28
:10BC43000000000000F85454545454D6000000007F
:10BC53006E0000000000DC6242424242E700000046
:10BC6300006F000000000018244242422418000024
:10BC730000007000000000DC62424242427C40E06F
:10BC830000000071000000007C848484848C7404B0
:10BC93000E000000720000000000EE322020202081
:10BCA300F8000000007300000000003C444038042A
:10BCB300447800000000740000000010107C101095
:10BCC3001010100C000000750000000000C6424276
:10BCD3004242463B00000000760000000000E742BD
:10BCE300242428101000000000770000000000D674
:10BCF3005454542828280000000078000000000055
:10BD03006E24181818247600000000790000000043
:10BD1300E742242428181010E00000007A000000F5
:10BD230000007E44081010227E000000007B00000B
:10BD330018101010101020101010101018007C0094
:10BD43001010101010101010101010101010107D83
:10BD530000003010101010100810101010103000D8
:10BD63007E0000000000000062928C0000000000D2
:10BD73000000C9EE400027FE240401208118560864
:10BD83005040104027FC2040C0E04158464E5844E4
:10BD930040404040DBDA0000120412441244FE44E7
:10BDA300124412441244124412443A44C444044414
:10BDB300080410040000CEB008400C40084017FCF3
:10BDC300104033FC3040504097FC10441044104462
:10BDD3001044105410481040C7B6010021083FF822
:10BDE3000000244024407E7C248425283C202420F9
:10BDF30024503C48248E25040200BFC606087888D8
:10BE030008480848FE0818881C482A48280E48781D
:10BE13008B8808080808080808080808BCBC102014
:10BE230010201020FDFE1020142019FC3108D088AA
:10BE33001090106010601090110E56042000B5E7AA
:10BE43000100010001003FF8210821083FF8210803
:10BE5300210821083FF821080102010200FE000029
:10BE6300D7D300003FF00020004000800100010014
:10BE73000104FFFE010001000100010001000500B3
:10BE83000200D3D0010001007FFE020004000FF086
:10BE9300181028104FF0881008100FF008100890A1
:10BEA30008700820CFDE0000FBF8920893F8A20880
:10BEB300A20893F88A808A48AA509220822082108E
:10BEC300828E83048200B9AB000004400640044024
:10BED300082008101018220E430402000420081042
:10BEE30011F83F1810100000CBBE00003FFC000407
:10BEF30000047FE4000400043FC4204420443FC402
:10BF030020442004001400080000C9E408081008B5
:10BF13003F0821083FFE21083F08214821287F28A8
:10BF2300052809081108210845280210C6B508008C
:10BF330008FE4E20484048FCFE8400A408A44AA4FE
:10BF43004AA484A4085010482086C3020000BFA856
:10BF53000100010001FC0100010001007FFE01005E
:10BF63000100014001300118010C0108010001002A
:10BF7300BDC92108320827C8445057DEF47417D4CA
:10BF8300211447D4F21403881A88E49404940AA66B
:10BF93001144B7D102403FF802483FF822403FFE28
:10BFA3000442084A1FF4681009100910091002C05E
:10BFB3000C383010CFB5007C3F80022004200840AD
:10BFC3001F8003200C103FF8108C04A008901088E9
:10BFD300208442840100CDB31040102023FE204072
:10BFE3004440F888090413FE20947C90009000904C
:10BFF3001D12E112020E0400D3E0010001000280D1
:10C00300046008103FFEC10401003FFC0100114021
:10C0130019301118211045000200B6EE100008FE79
:10C023007F9051201EFE228254820C9212923E92E5
:10C03300E29222AA22243E4221820000BAC51FF0C6
:10C043001010101010101FF00000FFFE0800080071
:10C053001FF0081000100010011000A00040D4AA27
:10C0630000001FF80000000000007FFE04400440B1
:10C07300044004400840084010422042403E000073
:10C08300B3F51000080008047EFE042408241224DB
:10C093003424582494241244104410841114120894
:10C0A3000000CABC1020183010201048FC8425FE64
:10C0B3002484440044FC288418841484228442FC8D
:10C0C30080840000BBAF08800C800888108C109817
:10C0D30030B050E090C0118012801480108410841E
:10C0E3001084107C0000CAA7010009000900110098
:10C0F3001FF82100410001007FFE01000280024081
:10C1030004200830101C2008B0DC00403E602240B0
:10C1130022802AFE2B882A882A882A500850142035
:10C12300122023502288410E0204D6D801F03F008A
:10C133000100FFFE01001FF011101FF011101FF08E
:10C1430001003FF801000100FFFE0000C6F40100FA
:10C1530000C000801FFC100410041FFC100010001E
:10C1630017FC14042404240447FC84040000D6D0E0
:10C173000100010021083FFC2108210821082108B2
:10C1830021083FF82108010001000100010001001E
:10C19300B6C10040404033FC204007FE0104E4A840
:10C1A30022A0222027FE20202050288831042206A6
:10C1B3000404C7EB004047FC304023F8004007FE6F
:10C1C300F00013F8120813F8120813F816081A08E7
:10C1D30012280210CBA23F822082209220923F920B
:10C1E300221222125FD2525252525252525252428F
:06C1F30093C2028A02045F
:10D8D300420056020349004C0931000004110011B3
:10D8E3000045004505300000041A401A220004FFD9
:10D8F300FFFFFFFFFF060000000000000000000024
:05D90300010203040510
:0BDAD100EF1FAC0670011E4C70F62227
:0BDA1B007C007E0012DA9C7F327E004F
:10DA2600AB07AA06EB1BAE0270011A4E60097F9582
:08DA36007E0012DAD180ED221E
:10DA7D00AD07AC06C2A5C2A4ECF580C2A3D2A3ED3E
:09DA8D00F580C2A3D2A3D2A522A8
:05DA5F00E0FEA3E0FF62
:10DA6400AD07AC06C2A5D2A4ECF580C2A3D2A3ED47
:09DA7400F580C2A3D2A3D2A522C1
:10DA3E0090000EE0FBA3E475F00112CF54A9F0FAAA
:04DA4E0012CEC4FF31
:0DDA5200C2A5D2A48F80C2A3D2A3D2A52268
:07DADC00901C00E0FF7E003A
:01DAE3002220
:06DA96007D077C007E000C
:0EDA9C00AB05AA0412DA7DAE02AF0302DA6413
:10C8C200C2A1C2A67F0A7E0012DA26D2A67D087C09
:10C8D200307FE37E0012DA9C7D127C007FE77E00CF
:10C8E20012DA9C7D317C127FEF7E0012DA9C7D0091
:10C8F2007C017F017E0012DA9C7D007C077F027E34
:10C902000012DA9C7D307C107F037E0012DA9CE4F8
:10C91200FDFC7F04FE12DA9C7D077C027F087E000C
:10C9220012DA9C7D007C077F097E0012DA9CE4FD0E
:10C93200FC7F0AFE12DA9CE4FDFC7F0CFE12DA9CFC
:10C94200E4FDFC7F0DFE12DA9CE4FDFC7F0FFE127B
:10C95200DA9C7DF07C007F107E0012DA9C7F11123F
:10C96200DA967D967C007F127E0012DA9CE4FDFC52
:10C972007F13FE12DA9C7FC87E0012DA267D907C3D
:10C98200147F107E0012DA9C7D277C027F1112DA5E
:10C992001D7D1D7F1212DA1B7D007C1A7F137E0023
:10C9A20012DA9C7D337C007F297E0012DA9C7D0E98
:10C9B2007F2B12DA1BE4FDFC7F20FE12DA9CE4FDE1
:10C9C200FC7F21FE12DA9C7F3012DA967D067C0211
:10C9D2007F317E0012DA9C7D067C057F327E00125A
:10C9E200DA9C7D047C077F357E0012DA9C7D037C15
:10C9F200127F367E0012DA9C7D077C007F377E0034
:10CA020012DA9CE4FDFC7F38FE12DA9C7D067C077C
:10CA12007F397E0012DA9C7D017C077F3C7E00120A
:10CA2200DA9C7D0F7C007F3D7E0012DA9CE4FDFCE7
:10CA32007F50FE12DA9C7DEF7C007F517E0012DA7D
:10CA42009CE4FDFC7F52FE12DA9C7D3F7C017F5309
:10CA52007E0012DA9C7D007CA77F607E0012DA9C49
:10CA62007D017C007F617E0012DA9CE4FDFC7F6A1E
:10CA7200FE12DA9C7D107C007F907E0012DA9C7D93
:10CA8200007C067F927E0012DA9C7D037C007F93FD
:10CA92007E0012DA9C7D107C017F957E0012DA9C6A
:10CAA200E4FDFC7F97FE12DA9CE4FDFC7F98FE1207
:10CAB200DA9C7D337C017F077E0012DA9C7F647EE4
:10CAC2000012DA26D2A190004A74FFF0A374E0F0BB
:0ACAD20090005874F8F0A3E4F0227D
:05D936002DFDE03CFCAA
:10D93B008D828C83AD07AC067F207E0012DA9CAE05
:10D94B0083AF82AD07AC067F217E0012DA9C7F226B
:05D95B007E0002DA7DF0
:10D77200900028EEF0A3EFF0A3ECF0A3EDF0A3EA03
:10D78200F0A3EBF0900028E0FCA3E0FD7F507E00C8
:10D7920012DA9C90002CE0FCA3E0FD7F517E001287
:10D7A200DA9C90002AE0FCA3E0FD7F527E0012DAB0
:10D7B2009C90002EE0FCA3E0FD7F537E0012DA9CD9
:10D7C200900028E0FEA3E0FFA3E0FCA3E0FD02D965
:01D7D2003B1B
:10D5C60090000CE4F0A374E7F074FFA3F0A3F07DE1
:0BD5D600C87BE67A007C007F787E00B6
:10D5E100900006EEF0A3EFF0A3ECF0A3EDF0A3EAB8
:04D5F100F0A3EBF0C8
:10D5F500C007A3E0FFA3E090002ECFF0A3EFF0D08B
:10D605000712D772900008E0FFA3E0900010CFF05A
:10D61500A3EFF090000CE0FEA3E0FFD3900011E033
:10D625009F900010E09E5034900006E0FEA3E0FBC2
:10D63500AA06C390000BE09B90000AE09A400D906B
:10D64500000E12DA5F0BBB00010A80E6900011E0C4
:0CD6550004F070BF900010E004F080B7FB
:01D6610022A6
:10D9870090000C7401F0A37440F0900058E0FFA3DE
:10D99700E090000ECFF0A3EFF07BF07A00E4FDFCFF
:05D9A700FFFE02D5E1C6
:08D7D300900003EEF0A3EFF05B
:10D7DB0090002E7401F0A3743FF07BEF7A00E4FD10
:10D7EB00FCFFFE12D772E4FDFCFFFE12D93BE49066
:10D7FB000005F0A3F0E4FBFA90000312DA5F0BBB19
:10D80B0000010ABA01F2BB40EF900006E004F07091
:10D81B0006900005E004F0C3900006E094F0900041
:06D82B0005E0940040CF6F
:01D8310022D4
:0ED23F00900012EEF0A3EFF0A3ECF0A3EDF0E0
:10D24D00E490001EF0A3F0A3F0A3F0A3F0A3F0A3CD
:10D25D00F0A3744FF0E490001EF0A3F090001EE0D8
:10D26D00FEA3E0FFC3944FEE9400502C12CEC4FDEC
:10D27D0090B83675F011EF12CF6AEE75F011A42546
:10D28D0083F583E4936D601090001FE004F070CC83
:10D29D0090001EE004F080C4900024E0FEA3E0FFA7
:10D2AD00C390001FE09F90001EE09E400302D3C379
:10D2BD00900012E0FAA3E0FBFFAE02C006C007A388
:10D2CD00E0FCA3E0FDEB2407FBE43AFA900014E048
:10D2DD00FEA3E0240FFFE43E90002EF0A3EFF0D06C
:10D2ED0007D00612D772E4900020F0A3F090002032
:10D2FD00E0FEA3E0FFC39410EE9400400302D3C3FD
:10D30D0090001EE0FCA3E090B83775F01112CF6AC3
:10D31D00EC75F011A42583F583E5822FF582E58365
:10D32D003EF583E493F9E4900022F0A3F0900022FF
:10D33D00E0FEA3E0FFC39408EE9400506874807E75
:10D34D0000A807088006CEA2E713CE13D8F8FFE990
:10D35D00FDEF5D6005900019800990001DE07008DB
:10D36D0090001B12DA5F802C900022E0FEA3E0FFFC
:10D37D00900013E02FFF900012E03ECF2401CF3438
:10D38D0000FE900020E0FCA3E0FD900015E0900071
:10D39D001412D936900023E004F07091900022E031
:10D3AD0004F002D33A900021E004F07006900020C2
:06D3BD00E004F002D2FAC8
:01D3C3002247
:0ECCD300900012EEF0A3EFF0A3ECF0A3EDF052
:10CCE100E490001EF0A3F0A3F0A3F0A3F0A3F09052
:10CCF1000026F0A37422F0E490001EF0A3F090004F
:10CD01001EE0FEA3E0FFC39422EE9400505112CE28
:10CD1100C4FD90BD7575F022EF12CF6AEE75F02259
:10CD2100A42583F583E493B5052590000112CEDD9A
:10CD3100FF90001EE0FCA3E090BD7675F02212CFBB
:10CD41006AEC75F022A42583F583E4936F6010905B
:10CD5100001FE004F070A790001EE004F0809F9097
:10CD61000026E0FEA3E0FFC390001FE09F90001E9D
:10CD7100E09E400302CEC3900012E0FAA3E0FBFF65
:10CD8100AE02C006C007A3E0FCA3E0FDEB240FFB4D
:10CD9100E43AFA900014E0FEA3E0240FFFE43E9091
:10CDA100002EF0A3EFF0D007D00612D772E4900066
:10CDB10020F0A3F0900020E0FCA3E0FD25E0FFECD3
:10CDC10033FE90001EE0FAA3E090BD7775F02212C9
:10CDD100CF6AEA75F022A42583F583E5822FF582D7
:10CDE100E5833EF583E493FAED25E0FFEC33FE9015
:10CDF100001EE0FCA3E090BD7875F02212CF6AEC32
:10CE010075F022A42583F583E5822FF582E5833E23
:10CE1100F583E493FFEAFE900024EEF0A3EFF0E443
:10CE2100900022F0A3F0900022E0FEA3E0FFC39463
:10CE310010EE9400506CE47E80A807088005CEC3F4
:10CE410013CE13D8F9FF900024E05EFEA3E05F4EFD
:10CE51006005900019800990001DE0700890001B8A
:10CE610012DA5F802C900022E0FEA3E0FF90001315
:10CE7100E02FFF900012E03ECF2401CF3400FE905E
:10CE81000020E0FCA3E0FD900015E090001412D911
:10CE910036900023E004F07006900022E004F002D6
:10CEA100CE27900021E004F07006900020E004F00D
:10CEB100C3900021E09410900020E0940050030200
:02CEC100CDB5ED
:01CEC300224C
:10D4DE00A3F0A37407F0A374E0F0E4A3F07D96FC30
:03D4EE007F2DFE91
:10D4F100900006EEF0A3EFF0A3ECF0A3EDF0A3EBA8
:10D50100F0A3EAF0A3E9F090000AE0FBA3E0FAA39C
:10D51100E0F912CEC4FF700302D5C5EFD394809019
:10D521000008E0FCA3E0FD404890000DE0FFA3E00F
:10D53100900019CFF0A3EFF090000FE0FFA3E0906F
:10D54100001BCFF0A3EFF0900011E090001DF090D0
:10D551000006E0FEA3E0FF12CCD3900007E0241008
:10D56100F0900006E03400F090000BE475F00280CA
:10D571004DA3E0FBA3E0FAA3E0F9A3E0FFA3E09051
:10D581000019CFF0A3EFF090000FE0FFA3E09000AF
:10D591001BCFF0A3EFF0900011E090001DF0900080
:10D5A10006E0FEA3E0FF12D23F900007E02408F05E
:10D5B100900006E03400F090000BE475F00112CF0A
:05D5C1003E02D5082226
:10C55E00900030EEF0A3EFF0A3ECF0A3EDF0A3EA21
:04C56E00F0A3EBF05B
:10C57200FFAE02E4FCFD7B807A967998F812D88FA0
:10C58200EF243090003CF0900034E0FEA3E0FFE4A2
:10C59200FCFD7B807A967998F812D88FAC00AD01B9
:10C5A200AE02AF037B407A42790F780012D88FEF48
:10C5B200243090003DF0900034E0FEA3E0FFE4FC64
:10C5C200FD7B807A967998F812D88FAC00AD01AED7
:10C5D20002AF037B407A42790F780012D88FAC0009
:10C5E200AD01AE02AF037BA07A867901780012D842
:10C5F2008FEF243090003EF0900034E0FEA3E0FF85
:10C60200E4FCFD7B807A967998F812D88FAC00AD65
:10C6120001AE02AF037B407A42790F780012D88FC5
:10C62200AC00AD01AE02AF037BA07A86790178003F
:10C6320012D88FAC00AD01AE02AF03E47B107A27B3
:10C64200F9F812D88FEF243090003FF0900034E0D8
:10C65200FEA3E0FFE4FCFD7B807A967998F812D87D
:10C662008FAC00AD01AE02AF037B407A42790F7806
:10C672000012D88FAC00AD01AE02AF037BA07A8668
:10C682007901780012D88FAC00AD01AE02AF03E49D
:10C692007B107A27F9F812D88FAC00AD01AE02AF49
:10C6A20003E47BE87A03F9F812D88FEF2430900084
:10C6B20040F0900034E0FEA3E0FFE4FCFD7B807AD2
:10C6C200967998F812D88FAC00AD01AE02AF037B19
:10C6D200407A42790F780012D88FAC00AD01AE02D9
:10C6E200AF037BA07A867901780012D88FAC00ADB7
:10C6F20001AE02AF03E47B107A27F9F812D88FACAF
:10C7020000AD01AE02AF03E47BE87A03F9F812D878
:10C712008FAC00AD01AE02AF03E47B64FAF9F8120C
:10C72200D88FEF2430900041F0900034E0FEA3E077
:10C73200FFE4FCFD7B807A967998F812D88FAC00E2
:10C74200AD01AE02AF037B407A42790F780012D876
:10C752008FAC00AD01AE02AF037BA07A867901787F
:10C762000012D88FAC00AD01AE02AF03E47B107AA9
:10C7720027F9F812D88FAC00AD01AE02AF03E47B0B
:10C78200E87A03F9F812D88FAC00AD01AE02AF031C
:10C79200E47B64FAF9F812D88FAC00AD01AE02AFB7
:10C7A20003E47B0AFAF9F812D88FEF2430900042A2
:10C7B200F0900034E0FEA3E0FFE4FCFD7B807A967B
:10C7C2007998F812D88FAC00AD01AE02AF037B406E
:10C7D2007A42790F780012D88FAC00AD01AE02AF69
:10C7E200037BA07A867901780012D88FAC00AD0164
:10C7F200AE02AF03E47B107A27F9F812D88FAC00AF
:10C80200AD01AE02AF03E47BE87A03F9F812D88FE8
:10C81200AC00AD01AE02AF03E47B64FAF9F812D8C2
:10C822008FAC00AD01AE02AF03E47B0AFAF9F81255
:10C83200D88FEB2430900043F0E4A3F090003BF05B
:10C8420090003BE0FFC394095075743C2FF582E4DD
:10C852003400F583E024D0700890003BE064087057
:10C862005690003BE0FB75F004A4FF900031E02FEE
:10C87200FF900030E035F0FEC007900032E0FCA3EC
:10C88200E0FD743C2BF9E43400FA7B01900036E0C1
:10C89200FFA3E090000DCFF0A3EFF0900038E0FF8F
:10C8A200A3E090000FCFF0A3EFF090003AE09000E9
:0FC8B20011F0D00702D4F190003BE004F0808138
:01C8C1002254
:06D6EE007A007C007E00C2
:10D6F400900006EEF0A3EFF0A3ECF0A3EDF0A3EAA4
:04D70400F0A3EBF0B3
:10D70800E4900011F0A3F090000CE0FEA3E0FFC34A
:10D71800900012E09F900011E09E504D900006E0AE
:10D72800FEA3E0FF900011E0FCA3E0FD900009E0FB
:10D738002DFD900008E03CFC12D93BE4FDFCD390A1
:10D74800000BE09D90000AE09C400D12DA3E12DAD0
:10D758003E0DBD00010C80E6900012E004F070A7B9
:09D76800900011E004F002D70F5B
:01D771002295
:10D08A0090000374FFF0A37400F0A3749EF0900064
:10D09A000CE4F0A37446F0900003E0F9A3E0FAA3CD
:10D0AA00E090000EC9F0A3EAF0A3E9F07BF07A0061
:10D0BA00E4FDFCFFFE12D6F490000CE4F0A3745DCC
:10D0CA00F0A374F8F0A3E4F07BEFFA7D46FCFFFED0
:10D0DA0012D5E17BFF7A00790390000D74FFF0A36B
:10D0EA0074E0F0A374F8F0A3E4F0A3F07D4AFC7FA7
:10D0FA0026FE12D4F190000C7401F0A3743FF0A341
:10D10A007407F0A374E0F07BEF7A007D5E7C00E4A4
:10D11A00FFFE12D5E190000374FFF0A37497F0A309
:10D12A007466F090000CE4F0A37414F0900003E02D
:10D13A00F9A3E0FAA3E090000EC9F0A3EAF0A3E98C
:10D14A00F07B787D6E7F7812D6EE7BFF7A007918B5
:10D15A00E490000DF0A3F0A37407F0A374E0F0E4E8
:10D16A00A3F07D86FC7F8CFE12D4F190000374FF3D
:10D17A00F0A37483F0A374DEF090000CE4F0A374BF
:10D18A0032F0900003E0F9A3E0FAA3E090000EC9A0
:10D19A00F0A3EAF0A3E9F07B327DB47F0F12D6EE5A
:10D1AA0090000374FFF0A374AAF0A37426F0900011
:10D1BA000CE4F0A3741EF0900003E0F9A3E0FAA3D4
:10D1CA00E090000EC9F0A3EAF0A3E9F07B3C7A00F4
:10D1DA007DEC7C007F0A7E0012D6F412D5C6900040
:10D1EA000C7401F0A3740BF074FFA3F0A3F07DECB0
:10D1FA0012D5D77BFF7A007921E490000DF0A3F0D5
:10D20A00A37407F0A374E0F0E4A3F07DD0FC7F5090
:10D21A00FE12D4F17BFF7A007926E490000DF0A388
:10D22A00F0A37407F0A374E0F0E4A3F07DF4FC7FAC
:05D23A0050FE02D4F1DA
:0CDAB900EF4E6007EF1F70F81E80F52292
:10D9AC0075CBFC75CA6975CDFC75CC69C2AD75C8F3
:10D9BC0004EF1FAC0670011E4C600730CFFDC2CFC8
:05D9CC0080EFC2CA2239
:10D9090075CBDC75CA0075CDDC75CC00C2AD75C8A8
:10D9190004EF1FAC0670011E4C600F20CF08300ABF
:0DD92900FAC2CAC2CF22C2CF80E7C2CA2212
:10D9D100750808AD081508ED6016EE2EFEC295EF2C
:10D9E100339297EF2FFFA296E4334EFED29580E358
:04D9F100D295AF0616
:01D9F500220F
:0EDAAA00C2937FAA12D9D17FFF12D9D1D29395
:01DAB800224B
:0DD3C4007F647E0012D9AC7B007A007922D4
:0BD3D100900003EBF0A3EAF0A3E9F0EA
:10D3DC00E4900007F0900006F0900006E0FCC39487
:10D3EC0064501912DAAAEFB4F00374FDF07F0A7ED0
:10D3FC000012DAB9900006E004F080DDEC64FE6007
:10D40C000302D4DBC2937FBB12D9D1900006EFF09C
:10D41C00900003E0FBA3E0FAA3E0F9740112CF0A39
:10D42C00E4900006F0900003E0FBA3E0FAA3E0F91F
:10D43C0012CEC4FF900006E0C39F50457FFF12D967
:10D44C00D1900003E0FBA3E0FAA3E0F9A3E0FEF522
:10D45C0082758300EF12CF1C900007E0FF8E82755F
:10D46C00830012CEDDFEEF6E900007F012CEC4D317
:10D47C0094204005D2937F0122900006E004F080B6
:10D48C00A47F0A7E0012D9AC7FFF12D9D190000381
:10D49C00E0FBA3E0FAA3E0F9A3E0F582758300EFCB
:10D4AC0012CF1C7F0A7E0012D9ACD293900003E0FD
:10D4BC00FBA3E0FAA3E0F9A3E0F58275830012CE9A
:10D4CC00DDFF900007E0B507037F00227F01227F7C
:01D4DC00014E
:01D4DD00222C
:0DD832007BFF900000EBF0A3EAF0A3E9F00B
:0BD83F00900003EBF0A3EAF0A3E9F077
:10D84A00E4A3F0C2937FCC12D9D1E4FC900003E0A8
:10D85A00FBA3E0FAA3E0F912CEC4FEECC39E501A71
:10D86A00900006E0FE8C8275830012CEDDFFEE6F1B
:10D87A00900006F012D9D10C80D2900006E0FF1277
:04D88A00D9D1D2938B
:01D88E002277
:0CDAC500C2927F327E0012D909D2922258
:10CADC00E4789DF608F608F608767812D9F612DA9C
:10CAEC00C57FF47E0112D9AC12C8C2E4FFFE12D786
:10CAFC00D312D08A2094FD801D900000E0FBA3E0AF
:10CB0C00FAA3E0F990000112CEDDFF7823E6B50719
:10CB1C0005789CE660107A00796812D83212D3C47A
:10CB2C00789CA60780D3789EE664011846700302B1
:10CB3C00CCD22094FD7F507E0002CC072094E77865
:10CB4C00A0E624FE18E634FFC364809480503F7B3B
:10CB5C00FF7A00799C12D83F789CA6077BFF7A005D
:10CB6C00792B90000DE4F0741F12D4DE7FF47E015B
:10CB7C0012D9AC7BFF7A00793690000D7407F074F3
:10CB8C00E012D4DE789D760008760102CB32801D4F
:10CB9C00900000E0FBA3E0FAA3E0F990000112CEB4
:10CBAC00DDFF7823E6B50705789CE660107A0079FE
:10CBBC008E12D83212D3C4789CA60780D37BFF7A0E
:10CBCC0000797612D83412D3C4789CA60790000052
:10CBDC00E0FBA3E0FAA3E0F990000112CEDDFF78B0
:10CBEC0023E6B50705789CE660177BFF7A00799CF5
:10CBFC0012D83F789CA6077FF47E0112D9AC02CBE9
:10CC0C00487824E6FF7E00789FEEF608EFF6FF905A
:10CC1C00000674FFF0A37400F0A37442F0A3EEF0CE
:10CC2C00A3EFF07B007A00797C12C25E7BFF7A0066
:10CC3C00799C12D83F789CA6077F647E0012D9ACF1
:10CC4C007BFF7A007945E490000DF0A3F074FFA30C
:10CC5C00F0A3F0E4A3F07DD0FC7F7DFE12D4F17B39
:10CC6C00007A00797CE490000DF0A3F074FFA3F03F
:10CC7C00A3F0E4A3F07DF4FC7F7DFE12D4F17BFFE6
:10CC8C007A00794EE490000DF0A3F074FFA3F0A3AA
:10CC9C00F0E4A3F07DF4FC7FB4FE12D4F17FD07EDF
:10CCAC000712D9AC12D5C690000C7401F0A3740B0A
:10CCBC00F074FFA3F0A3F07BE67A007DEC12D5DBD9
:06CCCC0012D5C602CB48A0
:01CCD200223F
:10D9F600C2AD75C804758780759870758921758D57
:10DA0600FD858D8BD28EC2ABD2AFC2A8D288C2CAD8
:05DA1600D2ACC20A229F
:0300000002D662C3
:0CD66200787FE4F6D8FD7581A002D6A9FF
:10CEC400BB010689828A83E0225002E722BBFE026C
:09CED400E32289828A83E493229F
:10CEDD00BB010CE58229F582E5833AF583E022500A
:10CEED0006E92582F8E622BBFE06E92582F8E22254
:0DCEFD00E58229F582E5833AF583E493226E
:10CF0A00BB010689828A83F0225002F722BBFE0106
:02CF1A00F32200
:10CF1C00F8BB010DE58229F582E5833AF583E8F04B
:10CF2C00225006E92582C8F622BBFE05E92582C8F7
:02CF3C00F222DF
:10CF3E00C5F0F8A3E028F0C5F0F8E582158270027E
:06CF4E001583E038F0221B
:10CF5400A3F8E0C5F025F0F0E58215827002158390
:06CF6400E0C838F0E822ED
:10D88F00C2D5E830E70FB2D5E4C39BFBE49AFAE4C4
:10D89F0099F9E498F8EC30E717B2D512D8C512CF42
:10D8AF00B2E4C39BFBE49AFAE499F9E498F8800395
:10D8BF0012CFB230D50DE4C39FFFE49EFEE49DFD71
:04D8CF00E49CFC22B7
:0CCF6A00A42582F582E5F03583F58322D2
:10C1F900E5082406F582E43400F583E00508229079
:10C209000003300703900006E475F00112D04402E0
:10C21900CEC42000E97F2ED2008018EF540F24905D
:10C22900D43440D4FF30040BEF24BFB41A005003B8
:10C239002461FFE50960021509050CE50C7002058A
:10C249000B30070E900003E475F00112D044EF02A1
:10C25900CF0A02D9607403D2078003E4C207F50844
:10C2690090000312D05BE4F509F50BF50CE50960C4
:10C27900077F2012C23C80F5750AFFC201C200C2C5
:10C2890002C203C205C206C20812C208FF700D30FD
:10C2990007057F0012C24DAF0CAE0B22B4255FC259
:10C2A900D5C20412C208FF24D0B40A00501A75F08E
:10C2B9000A780930D50508B6FF0106C6A426F62076
:10C2C900D5047002D20380D924CFB41A00EF5004E8
:10C2D900C2E5D20402C44ED20180C6D20080C0D2C7
:10C2E9000280BCD2D580BAD20580B47F2012C23C6C
:10C2F9002002077401B5090040F112C1F9FF12C209
:10C309003C02C276D208D206809512C1F9FB12C14D
:10C31900F9FA12C1F9F94A4B7006791F7AC57BFF00
:10C3290020022EE509602A7E008E8275830012CED6
:10C33900DD60060EEE650A70F0C2D5EBC0E0EAC01A
:10C34900E0E9C0E0EE12C495D0E0F9D0E0FAD0E01F
:10C35900FB12CEC4FF60AAEBC0E0EAC0E0E9C0E08E
:10C3690012C23CD0E02401F9D0E03400FAD0E0FB5D
:10C37900E50A0460DCD50AD980877BFF7AC4799104
:10C38900D202809C791080027908C206C20880080E
:10C39900D2D5790A8004790AC2D5E50A047002F572
:10C3A9000AE4FAFDFEFF12C1F9FC7B082001131211
:10C3B900C1F9FD7B1030000A12C1F9FE12C1F9FF63
:10C3C9007B20EC3382D592D55013C3E43000069F0D
:10C3D900FFE49EFEE42001039DFDE49CFCE4CBF810
:10C3E900C201EC700CCFCECDCCE824F8F870F38004
:10C3F90017C3EF33FFEE33FEED33FDEC33FCEB33C4
:10C40900FB994002FB0FD8E9EB300105F8D0E0C4F5
:10C4190048B201C0E00AEC4D4E4F78207B0070C253
:10C42900EAB50A0040BCC0E012C497D0F0D0E020C1
:10C439000104C4C0E0C4B201C0F012C225D0F0D5D5
:10C44900F0EB02C27612D064C31353C38D58C2E411
:10C459004CC2E042C3914FC39944C39949C2F943BD
:08C46900C39F55C38346C38342
:10C4710045C38347C53F50C2E82DC2EC2EC30F2BE5
:10C48100C2F023C30D20C5282AC2A8480000C30753
:10C491003F3F3F00790AA2D5200314300509B910A6
:10C4A100020404B9080104A2D520060250010420A7
:10C4B10002689202B509005034C0E07F20300319B0
:10C4C1007F30A20272067205500F12C4EEC202C280
:10C4D10006C205C2087F30800F300503E9C0E012B3
:10C4E100C23C300503D0E0F9D0E0B509CC300517E6
:10C4F1007F30B9100C12C23C7F583004077F78801E
:10C5010003B9080312C23C3002057F2D02C23C7FF1
:10C51100202008F87F2B2006F322920280CF286E7C
:10C52100756C6C2900D20112C1F93001F8C2017891
:10C531000930D50108F602C2A82D5043495812C14D
:10C54100F92403B405004001E490C53A9312C22DC9
:0DC55100743A12C22DD20375090402C38D85
:10D66E0002CADCE493A3F8E493A34003F68001F22C
:10D67E0008DFF48029E493A3F85407240CC8C333BD
:10D68E00C4540F4420C8834004F456800146F6DF8C
:10D69E00E4800B010204081020408090D8D3E47E71
:10D6AE00019360BCA3FF543F30E509541FFEE49381
:10D6BE00A360010ECF54C025E060A840B8E493A348
:10D6CE00FAE493A3F8E493A3C8C582C8CAC583CA73
:10D6DE00F0A3C8C582C8CAC583CADFE9DEE780BE2B
:01D90800001E
:10CF760075F008758200EF2FFFEE33FECD33CDCC72
:10CF860033CCC58233C5829BED9AEC99E5829840F5
:10CF96000CF582EE9BFEED9AFDEC99FC0FD5F0D6D2
:10CFA600E4CEFBE4CDFAE4CCF9A88222B800C1B9FC
:10CFB6000059BA002DEC8BF084CFCECDFCE5F0CB3A
:10CFC600F97818EF2FFFEE33FEED33FDEC33FCEB73
:10CFD60033FB10D703994004EB99FB0FD8E5E4F92E
:10CFE600FA227818EF2FFFEE33FEED33FDEC33FC1B
:10CFF600C933C910D7059BE99A4007EC9BFCE99A0F
:10D00600F90FD8E0E4C9FAE4CCFB2275F010EF2F53
:10D01600FFEE33FEED33FDCC33CCC833C810D70753
:10D026009BEC9AE899400AED9BFDEC9AFCE899F88E
:0ED036000FD5F0DAE4CDFBE4CCFAE4C8F92221
:10D04400F8E0FBA3A3E0F925F0F0E5821582700275
:07D054001583E0FA38F02219
:09D05B00EBF0A3EAF0A3E9F022D6
:10D06400D083D082F8E4937012740193700DA3A35B
:10D0740093F8740193F5828883E47374029368606F
:06D08400EFA3A3A380DF6F
:10D96000EFB40A07740D12D96B740A309811A89994
:10D97000B8130CC2983098FDA899C298B811F63027
:07D9800099FDC299F59922FF
:00000001FF
